:04000000F2EF24F007
:08000800056ED8CF06F0E0CF31
:1000100007F00001E9CF0DF0EACF08F0E1CF09F0D9
:10002000E2CF0AF0D9CF0BF0DACF0CF0F3CF14F017
:10003000F4CF15F0FACF16F000C00FF001C010F0A9
:1000400002C011F003C012F004C013F09DA62CEF03
:1000500000F09EB693EF11F0A0AA32EF00F0A1BA23
:1000600047EF11F00FC000F010C001F011C002F016
:1000700012C003F013C004F00DC0E9FF08C0EAFF8E
:10008000088E09C0E1FF0AC0E2FF0BC0D9FF0CC017
:10009000DAFF14C0F3FF15C0F4FF16C0FAFF0550D5
:1000A00007C0E0FF06C0D8FF1000F76ABA0FF66E6F
:1000B000000EF7220900F55012000003FFFFFFFFBA
:1000C000FFFFFFFFFFFFFFFFFFFF08AE03D0F2CFF0
:1000D0000EF0F29EF76AEC0FF66E000EF7220900A2
:1000E000F55008AE02D00EBEF28E1200400008009D
:1000F0000000000000000000000000000000000000
:10010000000000000000000000000000F76A1C0F63
:10011000F66E010EF7220900F55012000600FF09E5
:1001200001A101190129081580257F75089508810D
:100130000819012908750895089108C0F76A4C0F3D
:10014000F66E010EF7220900F55012000000F76A62
:100150005E0FF66E010EF7220900F5501200200026
:10016000F76A700FF66E010EF7220900F5501200C3
:1001700009022900010100C0320904000002030045
:100180000000092100010001222000070581030869
:1001900000010705010308000100F76AAA0FF66EC7
:1001A000010EF7220900F55012000100F76ABC0F9A
:1001B000F66E010EF7220900F55012001200F76AE0
:1001C000CE0FF66E010EF7220900F5501200120153
:1001D0001001000000406104231000010102000131
:1001E000F76AF00FF66E010EF7220900F5501200C3
:1001F0000403090408035400440045002C03540080
:1002000065006300680044006500730069006700D2
:100210006E002000540044002D0043004D005000AB
:100220002000300032003300F2CF0EF0F29EF76A69
:10023000420FF66E020EF7220900F5500EBEF28E46
:100240001200000000000000005F0000000700072F
:1002500000147F147F14242A7F2A12231308646257
:1002600036495522500005030000001C22410000C1
:1002700041221C0014083E081408083E08080050DB
:10028000300000080808080800606000002010081E
:1002900004023E5149453E00427F400042615149BF
:1002A000462141454B311814127F102745454539E9
:1002B0003C4A494930017109050336494949360626
:1002C0004949291E00363600000056360000081441
:1002D0002241001414141414004122140802015184
:1002E0000906324979413E7E1111117E7F49494903
:1002F000363E414141227F4141221C7F49494941CB
:100300007F090909013E4149497A7F0808087F00B1
:10031000417F41002040413F017F081422417F403E
:100320004040407F020C027F7F0408107F3E414125
:10033000413EF2CF0EF0F29EF76A4C0FF66E030EBE
:10034000F7220900F5500EBEF28E12007F0909094E
:10035000063E4151215E7F091929464649494931E6
:1003600001017F01013F4040403F1F2040201F3FCF
:100370004038403F63140814630708700807615150
:10038000494543007F4141000204081020004141DB
:100390007F0004020102044040404040000102048A
:1003A0000020545454787F4844443838444444200E
:1003B000384444487F3854545418087E0901020CCC
:1003C0005252523E7F0804047800447D4000204091
:1003D000443D007F1028440000417F40007C041809
:1003E00004787C0804047838444444387C14141499
:1003F00008081414187C7C08040408485454542039
:10040000043F4440203C4040207C1C2040201C3CB9
:100410004030403C44281028440C5050503C446428
:10042000544C44000836410000007F000000413673
:10043000080010080810087846414678F2CF0EF000
:10044000F29EF76A560FF66E040EF7220900F55079
:100450000EBEF28E1200000080C0E0F0F0F8FCFC4E
:10046000FCFCFEFEF1F1FEFEFCFCFCFCF8F0F0E012
:10047000C08000001824E7E7FFFFFFFFFFFFFFFF3A
:10048000FFFFFFFFFFFFFFFFFFFFFFFFFFFFE7E7AC
:10049000241800000103070F0F1F3F3F3F3F7F7FDE
:1004A0008F8F7F7F3F3F3F3F1F0F0F0703010000EC
:1004B000F2CF0EF0F29EF76ACA0FF66E040EF72224
:1004C0000900F5500EBEF28E1200000080C0E0F070
:1004D000F0F8FCFCFCCCF6FA0101FAF6CCFCFCFCD2
:1004E000F8F0F0E0C08000001824E7E7FFFFFFFF0E
:1004F000FFFFFFFFFFFF0000FFFFFFFFFFFFFFFF0A
:10050000FFFFE7E7241800000103070F0F1F3F3F1D
:100510003F3F7F7F80807F7F3F3F3F3F1F0F0F0721
:1005200003010000F2CF0EF0F29EF76A3E0FF66E66
:10053000050EF7220900F5500EBEF28E12000000E3
:1005400080C0E0F0F0F8FCFCFCFCFEFE0303FEFEC5
:10055000FCFCFCFCF8F0F0E0C08000001824E7E7A9
:10056000FFFFFFFFFFFFFFFFFFFF0000FFFFFFFF99
:10057000FFFFFFFFFFFFE7E7241800000103070F5D
:100580000F1F3F3F3F336F5F80805F6F333F3F3FC1
:100590001F0F0F0703010000F2CF0EF0F29EF76A63
:1005A000B20FF66E050EF7220900F5500EBEF28E60
:1005B0001200000080C0E0F0F0F8FCFCFCFCFEFE45
:1005C000F1F1FEFEFCFCFCFCF8F0F0E0C080000065
:1005D0001824C3A56666E7E7E7E7E7E7E7E7E7E7A5
:1005E000E7E7E7E7E7E7E7E7E7E7E7E724180000FB
:1005F0000103070F0F1F3F3F3F3F7F7F8F8F7F7F9D
:100600003F3F3F3F1F0F0F0703010000F2CF0EF0E7
:10061000F29EF76A260FF66E060EF7220900F550D5
:100620000EBEF28E1200000080C0E0F0F0F8FCFC7C
:10063000FCFCFEFEF1F1FEFEFCFCFCFCF8F0F0E040
:10064000C08000001824E7E7E7E7E7E7E7E7E7E728
:10065000E7E7E7E7E7E7E7E7E7E7E7E76666A5C392
:10066000241800000103070F0F1F3F3F3F3F7F7F0C
:100670008F8F7F7F3F3F3F3F1F0F0F07030100001A
:10068000F2CF0EF0F29EF76A9A0FF66E060EF72280
:100690000900F5500EBEF28E1200000080C0E0F09E
:1006A000F0F8FCFCFCFCFEFEF1F1FEFEFC6C2C8C78
:1006B000C800F0E0C08000001824E7E7FFFFFFFF5C
:1006C000FFFF7F3F9FCFE7F7F3F9FCFEFFFFFFFE41
:1006D000FFFFE7E7241800000103070F0713393C69
:1006E0003E3F7F7F8F8F7F7F3F3F3F3F1F0F0F0733
:1006F00003010000F2CF0EF0F29EF76A0E0FF66EC5
:10070000070EF7220900F5500EBEF28E120000000F
:1007100080C0E0F0F0C89C3C7CFCFEFEF1F1FEFEE7
:10072000FCFCFCFCF8F0F0E0C08000001824E7E7D7
:10073000FFFFFFFFFFFFFEFCF9F3F7E7CF9F3F7FCF
:10074000FFFFFF7FFFFFE7E7241800000103070F0B
:100750000F1F3F3F3F3F7F7F8F8F7F7F3736343183
:1007600013000F0703010000F2CF0EF0F29EF76AAC
:10077000820FF66E070EF7220900F5500EBEF28EBC
:100780001200000080C0E0F0F0F8FCFCFCFCFEFE73
:10079000F1F1FEFEFC7C3C9CC8E0F0E0C080000073
:1007A0001824E7E7FFFF7FFFFFFF7F3F9FCFE7F7BB
:1007B000F3F9FCFEFFFFFFFFFFFFE7E7241800004F
:1007C0000103070F00133134363F7F7F8F8F7F7F08
:1007D0003F3F3F3F1F0F0F0703010000F2CF0EF016
:1007E000F29EF76AF60FF66E070EF7220900F55033
:1007F0000EBEF28E1200000080C0E0F000C88C2C0B
:100800006CECFEFEF1F1FEFEFCFCFCFCF8F0F0E00E
:10081000C08000001824E7E7FFFFFEFFFFFFFEFC9B
:10082000F9F3F7E7CF9F3F7FFFFFFFFFFFFFE7E70A
:10083000241800000103070F0F1F3F3F3F3F7F7F3A
:100840008F8F7F7F3F3E3C39130F0F07030100005E
:10085000F2CF0EF0F29EF76A6A0FF66E080EF722DC
:100860000900F5500EBEF28E1200000080C0E0F0CC
:10087000F0F8FCFCFCFCFEFEFFFFF63A0AC0F0CCF0
:10088000F8F0F0E0C08000001824E7E7FFFFFFFF6A
:10089000FFFFFFFFFFFF1F87E0FCFFFFFFFFFFFFE2
:1008A000FFFFE7E7241800000103070F0F1F3F3F7A
:1008B0003F0F43708C8F7F7F3F3F3F3F1F0F0F07DE
:1008C00003010000F2CF0EF0F29EF76ADE0FF66E23
:1008D000080EF7220900F5500EBEF28E120000003D
:1008E00080C0E0F0F0F8FCFCFCFCFEFEF1F1FEFE46
:1008F000FCFCFCFC58501020008000001824E7E7A6
:10090000FF7F7F3F3F9F9FCFCFE7E7F3F3FBF9FDEB
:10091000FCFEFEFEFFFFFCFF3C1800000100040E81
:100920000E1F3F3F3F3F7F7F8F8F7F7F3F3F3F3F88
:100930001F0F0F0701010000F2CF0EF0F29EF76AC1
:10094000520FF66E090EF7220900F5500EBEF28E18
:1009500012000000804060F0F0F8FCFCFCFCFEFEA1
:10096000F1F1FEFEFCFCFCFCF8F0F0E0C0800000C1
:100970001824E7E6FEFCFCFDF9F9F3F3F7E7E7EFEF
:10098000CFCF9F9FBF3F3F7F7FDF3FFF3C180000DF
:100990000103070F0F1F3F3F3F3F7F7F8F8F7F7FF9
:1009A0003F3F3F3F1B0A0A0400010000F2CF0EF058
:1009B000F29EF76AC60FF66E090EF7220900F5508F
:1009C0000EBEF28E1200000080C0E0F0F0F8F8F0E9
:1009D000C08C1E7EF1F1FEFEFCFCFCFCF8F0F0E0A9
:1009E000C08000001824E7E7FFFFFFFFFFFFFFFFC5
:1009F000FEF8E1871F7FFFFFFFFFFFFFFFFFE7E735
:100A0000241800000103070F0F1F3F3F3F3F7F7F68
:100A1000FFEF4E5841070F311F0F0F070301000072
:100A2000F2CF0EF0F29EF76A3A0FF66E0A0EF72238
:100A30000900F5500EBEF28E1200000080C0E0F0FA
:100A4000F0F8FCFCFCFCFEFEF1F1FE3E0CC0F0FCFC
:100A5000F8F0F0E0C08000001824E7E7FFFFFFFF98
:100A6000FFFFFFFFFFFF1F87E0FCFFFFFFFFFFFF10
:100A7000FFFFE7E7241800000103070F0F1F3F3FA8
:100A8000210F4350DCEF7F7F3F3F3F3F1F0F0F079A
:100A900003010000F2CF0EF0F29EF76AAE0FF66E81
:100AA0000A0EF7220900F5500EBEF28E1200000069
:100AB00080C0E0F0F0F8FCFCFCFCFEFEF1F1FEFE74
:100AC000FCFCFCFC7870302080800000183CFF3F6C
:100AD000FF7F7F3F3F9F9FCFCFE7E7F3F3FBF9FD1A
:100AE000FCFEFEFEFFFFE7E7241800000100000AFD
:100AF0000A1F3F3F3F3F7F7F8F8F7F7F3F3F3F3FBB
:100B00001F0F0F0701010000F2CF0EF0F29EF76AEF
:100B1000220FF66E0B0EF7220900F5500EBEF28E74
:100B200012000000004020B0B0F8FCFCFCFCFEFE0F
:100B3000F1F1FEFEFCFCFCFCF8F0F0E0C0800000EF
:100B4000183CFEF8F6FCFCFDF9F9F3F3F7E7E7EFE4
:100B5000CFCF9F9FBF3F3F7F7FFFE7E72418000075
:100B60000103070F0F1F3F3F3F3F7F7F8F8F7F7F27
:100B70003F3F3F3F1F0E0E0400010000F2CF0EF07A
:100B8000F29EF76A960FF66E0B0EF7220900F550EB
:100B90000EBEF28E1200000080C0E0F0F0F8FC8083
:100BA000E0C2823677FFFEFEFCFCFCFCF8F0F0E0D1
:100BB000C08000001824E7E7FFFFFFFFFFFFFFFFF3
:100BC000FFFEF8E1871F7FFFFFFFFFFFFFFFE7E763
:100BD000241800000103070F0F1F3F3F3F3F7F7F97
:100BE0008F8F7F7E3821073F1F0F0F070301000003
:100BF000F2CF0EF0F29EF76A0A0FF66E0C0EF72295
:100C00000900F5500EBEF28E12007F7F0101010F28
:100C10000101013F0101010F0101017F7F0101017C
:100C20000F0101013F0101010F0101017F7FF2CF9F
:100C30000EF0F29EF76A480FF66E0C0EF7220900CE
:100C4000F5500EBEF28E12000101011111FF8081DC
:100C5000819191FF0181819191FF8080808888FF3F
:100C6000F2CF0EF0F29EF76A7A0FF66E0C0EF722B4
:100C70000900F5500EBEF28E12007072655F696E4B
:100C8000697431200A0D0000F2CF0EF0F29EF76A6F
:100C9000A20FF66E0C0EF7220900F5500EBEF28E72
:100CA00012004272696768746E6573730000F2CF58
:100CB0000EF0F29EF76AC80FF66E0C0EF7220900CE
:100CC000F5500EBEF28E120041646A757374000016
:100CD000F2CF0EF0F29EF76AEA0FF66E0C0EF722D4
:100CE0000900F5500EBEF28E12005465636844652B
:100CF0007369676E2E626500F2CF0EF0F29EF76A9E
:100D0000120FF66E0D0EF7220900F5500EBEF28E90
:100D10001200706F73745F696E697431200A0D0080
:100D2000F2CF0EF0F29EF76A3A0FF66E0D0EF72232
:100D30000900F5500EBEF28E1200566F703D202550
:100D400075200000F2CF0EF0F29EF76A5E0FF66E8D
:100D50000D0EF7220900F5500EBEF28E1200202073
:100D60002020202020202020202020200000F2CF42
:100D70000EF0F29EF76A880FF66E0D0EF72209004C
:100D8000F5500EBEF28E1200202020202020000000
:100D9000F2CF0EF0F29EF76AAA0FF66E0D0EF72252
:100DA0000900F5500EBEF28E12000D0A2078615F28
:100DB0006D61785F63616C69623D20256C75000030
:100DC000F2CF0EF0F29EF76ADA0FF66E0D0EF722F2
:100DD0000900F5500EBEF28E12000D0A2078625FF7
:100DE0006D61785F63616C69623D20256C75000000
:100DF000F2CF0EF0F29EF76A0A0FF66E0E0EF72291
:100E00000900F5500EBEF28E12000D0A2079615FC6
:100E10006D61785F63616C69623D20256C750000CF
:100E2000F2CF0EF0F29EF76A3A0FF66E0E0EF72230
:100E30000900F5500EBEF28E12000D0A2079625F95
:100E40006D61785F63616C69623D20256C7500009F
:100E5000F2CF0EF0F29EF76A6A0FF66E0E0EF722D0
:100E60000900F5500EBEF28E12000D0A2078615F67
:100E70006469665F63616C69623D20256C75000082
:100E8000F2CF0EF0F29EF76A9A0FF66E0E0EF72270
:100E90000900F5500EBEF28E12000D0A2078625F36
:100EA0006469665F63616C69623D20256C75000052
:100EB000F2CF0EF0F29EF76ACA0FF66E0E0EF72210
:100EC0000900F5500EBEF28E12000D0A2079615F06
:100ED0006469665F63616C69623D20256C75000022
:100EE000F2CF0EF0F29EF76AFA0FF66E0E0EF722B0
:100EF0000900F5500EBEF28E12000D0A2079625FD5
:100F00006469665F63616C69623D20256C750000F1
:100F1000F2CF0EF0F29EF76A2A0FF66E0F0EF7224E
:100F20000900F5500EBEF28E12000D0A0D0A54652E
:100F30006D703D2020202025322E31664320202553
:100F4000332E316646200D0A0000F2CF0EF0F29EDD
:100F5000F76A640FF66E0F0EF7220900F5500EBE09
:100F6000F28E12000D0A20586120256C7500F2CF18
:100F70000EF0F29EF76A880FF66E0F0EF722090048
:100F8000F5500EBEF28E12000D0A20586220256C1C
:100F90007500F2CF0EF0F29EF76AAC0FF66E0F0EF0
:100FA000F7220900F5500EBEF28E12000D0A2059EC
:100FB0006120256C7500F2CF0EF0F29EF76AD00F1B
:100FC000F66E0F0EF7220900F5500EBEF28E1200DB
:100FD0000D0A20596220256C7500F2CF0EF0F29EAA
:100FE000F76AF40FF66E0F0EF7220900F5500EBEE9
:100FF000F28E12000D0A2058613220256C75000017
:10100000F2CF0EF0F29EF76A1A0FF66E100EF7226C
:101010000900F5500EBEF28E12000D0A2058623201
:1010200020256C750000F2CF0EF0F29EF76A400F9B
:10103000F66E100EF7220900F5500EBEF28E120069
:101040000D0A2059613220256C750000F2CF0EF098
:10105000F29EF76A660FF66E100EF7220900F55041
:101060000EBEF28E12000D0A2059623220256C75D8
:101070000000F2CF0EF0F29EF76A8C0FF66E100EA3
:10108000F7220900F5500EBEF28E12000D0A204321
:101090006F6D7061737320583D20254C64200000F3
:1010A000F2CF0EF0F29EF76ABA0FF66E100EF7222C
:1010B0000900F5500EBEF28E12000D0A20436F6D2E
:1010C0007061737320593D20254C64200D0A000087
:1010D000F2CF0EF0F29EF76AEA0FF66E100EF722CC
:1010E0000900F5500EBEF28E1200436F6D706173F1
:1010F000733D202025332E3066200A0D0000F2CFEC
:101100000EF0F29EF76A180FF66E110EF722090024
:10111000F5500EBEF28E12002D2D2D00F2CF0EF0E6
:10112000F29EF76A360FF66E110EF7220900F5509F
:101130000EBEF28E1200204E2000F2CF0EF0F29E74
:10114000F76A540FF66E110EF7220900F5500EBE25
:10115000F28E12004E4E4500F2CF0EF0F29EF76A6C
:10116000720FF66E110EF7220900F5500EBEF28EC8
:101170001200204E4500F2CF0EF0F29EF76A900F5B
:10118000F66E110EF7220900F5500EBEF28E120017
:10119000454E4500F2CF0EF0F29EF76AAE0FF66EA6
:1011A000110EF7220900F5500EBEF28E12002045F6
:1011B0002000F2CF0EF0F29EF76ACC0FF66E110E01
:1011C000F7220900F5500EBEF28E1200455345007D
:1011D000F2CF0EF0F29EF76AEA0FF66E110EF722CA
:1011E0000900F5500EBEF28E120020534500F2CFDA
:1011F0000EF0F29EF76A080FF66E120EF722090043
:10120000F5500EBEF28E120053534500F2CF0EF091
:10121000F29EF76A260FF66E120EF7220900F550BD
:101220000EBEF28E120020532000F2CF0EF0F29E7E
:10123000F76A440FF66E120EF7220900F5500EBE43
:10124000F28E120053535700F2CF0EF0F29EF76A5F
:10125000620FF66E120EF7220900F5500EBEF28EE6
:10126000120020535700F2CF0EF0F29EF76A800F63
:10127000F66E120EF7220900F5500EBEF28E120025
:1012800057535700F2CF0EF0F29EF76A9E0FF66E9C
:10129000120EF7220900F5500EBEF28E12002057F2
:1012A0002000F2CF0EF0F29EF76ABC0FF66E120E1F
:1012B000F7220900F5500EBEF28E1200574E57006D
:1012C000F2CF0EF0F29EF76ADA0FF66E120EF722E8
:1012D0000900F5500EBEF28E1200204E5700F2CFDC
:1012E0000EF0F29EF76AF80FF66E120EF722090062
:1012F000F5500EBEF28E12004E4E5700F2CF0EF099
:10130000F29EF76A160FF66E130EF7220900F550DB
:101310000EBEF28E120054696C743D2020202020F5
:10132000253364200A0D0000F2CF0EF0F29EF76A1A
:10133000420FF66E130EF7220900F5500EBEF28E24
:101340001200526F6C6C3D20202020202533642039
:101350000A0D200A0D00F2CF0EF0F29EF76A700F10
:10136000F66E130EF7220900F5500EBEF28E120033
:101370000D0A2D2D3E2052656365697665642064F3
:101380006174613A20307825582030782558000063
:10139000F2CF0EF0F29EF76AAA0FF66E130EF72246
:1013A0000900F5500EBEF28E12000D0A436F6D70EB
:1013B0006173732063616C6962726174696F6E003E
:1013C000F2CF0EF0F29EF76ADA0FF66E130EF722E6
:1013D0000900F5500EBEF28E12000D0A2078615FF2
:1013E0006D61783D20256C750000F2CF0EF0F29E05
:1013F000F76A040FF66E140EF7220900F5500EBEC0
:10140000F28E12000D0A2078625F6D61783D202512
:101410006C750000F2CF0EF0F29EF76A2E0FF66E9A
:10142000140EF7220900F5500EBEF28E12000D0ABE
:101430002079615F6D61783D20256C750000F2CFE9
:101440000EF0F29EF76A580FF66E140EF72209009E
:10145000F5500EBEF28E12000D0A2079625F6D61AA
:10146000783D20256C750000F2CF0EF0F29EF76AF1
:10147000820FF66E140EF7220900F5500EBEF28EA2
:1014800012000D0A2078615F6469663D20256C7545
:101490000000F2CF0EF0F29EF76AAC0FF66E140E5B
:1014A000F7220900F5500EBEF28E12000D0A2078C8
:1014B000625F6469663D20256C750000F2CF0EF016
:1014C000F29EF76AD60FF66E140EF7220900F55059
:1014D0000EBEF28E12000D0A2079615F6469663DCE
:1014E00020256C750000F2CF0EF0F29EF76A000F17
:1014F000F66E150EF7220900F5500EBEF28E1200A0
:101500000D0A2079625F6469663D20256C750000D4
:10151000F2CF0EF0F29EF76A2A0FF66E150EF72242
:101520000900F5500EBEF28E120063616C696272A2
:101530006174696F6E206F6B2100F2CF0EF0F29E26
:10154000F76A540FF66E150EF7220900F5500EBE1D
:10155000F28E12000D0A0A55534220636F6E6E65BB
:10156000637465642C2077616974696E6720666FA7
:101570007220656E756D65726174696F6E2E2E2EA8
:101580000000F2CF0EF0F29EF76A9C0FF66E150E79
:10159000F7220900F5500EBEF28E12000D0A0A5510
:1015A000534220646973636F6E6E65637465642C67
:1015B0002077616974696E6720666F7220636F6E51
:1015C0006E656374696F6E2E2E2E0000F2CF0EF0E2
:1015D000F29EF76AE60FF66E150EF7220900F55037
:1015E0000EBEF28E12000D0A0A55534220656E752A
:1015F0006D6572617465642062792050432F484F95
:1016000053540000F2CF0EF0F29EF76A1E0FF66EF2
:10161000160EF7220900F5500EBEF28E12000D0ACA
:101620000A55534220756E656E756D6572617465FD
:10163000642062792050432F484F53542C20776107
:101640006974696E6720666F7220656E756D65726C
:101650006174696F6E2E2E2E00006D92699468A4DD
:1016600002D06894FCD752EF11F0400E0401016FD4
:10167000040E036F100E026F880E006F046B040ED1
:10168000076F500E066F0001000C70A002D0EDDF56
:101690007090689A5BEF11F06A6A689261EF11F0DE
:1016A000036A01013F51700FE96E0F0E0320EA6ECD
:1016B000EF6A3F51080DF350416BE96E040E41256E
:1016C000EA6EEF6A3F51080DF350416B406F040E14
:1016D0004027000E412340C1E9FF040E4125EA6E78
:1016E000EF6A0001000C010E01013E6F3E510F0830
:1016F00007E33EC13FF10001D3DF01013E2BF6D7E6
:101700000001000C0101346B34530AE1036A3451C7
:101710002B0FE96E000E0320EA6EEF6A342BF4D72C
:10172000206A010E216E1F6A0001000C689600D02D
:1017300000D000D0000C6A6A686A9F0E6B6E3D0E86
:10174000696E6E6AD0DFDEDF160E706E68A602D09C
:10175000EDDFFCD76D9889DF030E266E67EF11F081
:10176000698468986D826DEF11F0689C73EF11F0D9
:1017700039C127F0000CFF0E276E000C0101376BFA
:101780002A524CE037513F0849E32250FC0F35E222
:10179000040F000119EF0CF0036A2950F2CF39F160
:1017A000F29EB0EC00F0010139BFF28E386F25D007
:1017B000036A2950F2CF39F1F29E86EC00F0010164
:1017C00039BFF28E386F19D0036A2950F2CF39F140
:1017D000F29EF0EC00F0010139BFF28E386F0DD0AF
:1017E000036A2950F2CF39F1F29EDFEC00F00101DB
:1017F00039BFF28E386F01D00101292A2A063751EC
:10180000372B036A500F016E000E032201C0E9FF5F
:10181000040E0324EA6E38C1EFFFB2D72A5204E166
:101820003751400801E01F6A37C139F10001A0DFDC
:10183000000CE824F76AF7364D0FF66E180EF72203
:101840000A00F550FA6E0800F550F96E9817B017B7
:10185000C817E017296A226A04011351010A00011E
:1018600009E0030A0CE0010A0DE0220A25E0030A60
:101870004AE077D0120E2A6E030E226E74D0290E23
:101880002A6E71D0020E226E036A04011251230FD8
:10189000E96E000E0320EA6EEFCF29F0036A2950AB
:1018A000F2CF37F1F29E0001F0EC00F0010137BFFA
:1018B000F28E2A6E000157D0D89004011235036AC7
:1018C000F2CF37F1F29E0001D6EC00F00900F5CF1F
:1018D00003F0010137BFF28E296E293C01D010D0F0
:1018E000036A2950F2CF37F1F29E0001B0EC00F00C
:1018F000010137BFF28E2A6E000135D004D00101FC
:10190000000139DF3CD0D89004011435036AF2CFCE
:1019100037F1F29E00019EEC00F00900F5CF03F0D4
:10192000010137BFF28E296E293C01D017D0010E7C
:10193000226ED89004011435036AF2CF37F1F29E7B
:101940000001A7EC00F00900F5CF03F0010137BF5B
:10195000F28E2A6E000107D004D0010100010BDFD6
:101960000ED009DF0CD00401175305E12A50165D93
:1019700002E216C42AF0010E1F6E0001FFDE000C09
:101980000101365306E1040E266E0001ACDEE4D000
:101990000101050E266E040E396F900E386F010E90
:1019A000376F37510F08D8A0D7D037C13FF10001AA
:1019B00077DE01013A6B036A3751F2CF3EF1F29EB6
:1019C000000155EC00F001013EBFF28EFF085DE022
:1019D000040E3A6FD8903735036AF2CF3EF1F29E8B
:1019E000000165EC00F00900F5CF03F001013EBFF6
:1019F000F28E3B6F03C03CF13751080DF3503F6B43
:101A00003E6F010E3E25016E000E3F21036E01C0A8
:101A1000E9FF040E0324EA6E3BC1EFFF3751080DC6
:101A2000F3503F6B3E6F020E3E25016E000E3F21CC
:101A3000036E01C0E9FF040E0324EA6E39C1ECFF16
:101A4000ED5238C1EFFFD8903735036AF2CF3EF13F
:101A5000F29E000165EC00F00900F5CF03F00101F2
:101A60003EBFF28E382703503923880E3D6F3CB1BC
:101A70003D813CB33D833751080DF3503F6BE96E18
:101A8000040E3F25EA6E3DC1EFFF036A3751F2CFE6
:101A90003EF1F29E000155EC00F001013EBFF28ED6
:101AA000FF083CE03A833751080DF3503F6B3E6F1F
:101AB000040E3E27000E3F23020E3E25016E000E4F
:101AC0003F21036E01C0E9FF040E0324EA6E39C111
:101AD000ECFFED5238C1EFFFD8903735036AF2CFF3
:101AE0003EF1F29E000165EC00F00900F5CF03F035
:101AF00001013EBFF28E3827035039233751080DBC
:101B0000F3503F6B3E6F040E3E27000E3F233EC155
:101B1000E9FF040E3F25EA6E400EEF6E3A510608CB
:101B200002E10E0E3A6F036A3751F2CF3EF1F29E98
:101B3000000155EC00F001013EBFF28E0108D8A46F
:101B40003A89036A3751700FE96E0F0E0320EA6E6F
:101B50003AC1EFFF372B25D7000100EF0EF004014B
:101B6000115100010DE0010A15E0020A20E0060A09
:101B70002AE0030A31E00E0A31E0010A37E046D0DC
:101B800021C050F40401516B020E0101396F0001B4
:101B9000EFDD3ED00401122D07D0010E2116010108
:101BA000396B0001E5DD02D00001E5DD31D0040133
:101BB000122D06D021820101396B0001D9DD02D03E
:101BC0000001D9DD25D0020E1F6E12C428F00101DC
:101BD000396B0001CDDD1CD03DDE1AD020C050F4A1
:101BE000010E0101396F0001C3DD12D00401125151
:101BF00001080AE312C420F012C436F10001C0D675
:101C00000101396B0001B4DD000102D0B4DD00D068
:101C10005CEF0FF020C036F104011151000107E024
:101C20000A0A0EE0010A34E00D0A47E048D0040138
:101C3000506B516B020E0101396F000199DD41D0EB
:101C40000101365322E0010E365D036AF2CF37F10F
:101C5000F29E0001CDEC00F0010137BFF28E016E63
:101C60000401145DD8A002D001010FD0036A145101
:101C70002B0FE96E000E0320EA6EEFCF50F4010E39
:101C80000101396F000174DD02D0000174DD19D04B
:101C9000010136530FE0036A040114512B0FE96E62
:101CA000000E0320EA6E12C4EFFF0101396B000140
:101CB0005FDD02D000015FDD04D0CCDD02D05BDD52
:101CC00000D05CEF0FF00101379136BF3781369FAE
:101CD00037A113D0036A3651F2CF38F1F29E0001DA
:101CE00055EC00F0010138BFF28EFF0802E1000E52
:101CF00001D0010E016E13D012D0036A3651F2CF1B
:101D000038F1F29E000155EC00F0010138BFF28E6F
:101D1000FF0802E1000E01D0010E016E00D00001AB
:101D20000BEF0FF00101379136BF3781369F37A196
:101D300011D03651080DF350396B386F040E382727
:101D4000000E392338C1E9FF040E3925EA6E880EEA
:101D5000EF6E09D03651080DF350396BE96E040E61
:101D60003925EA6EEF6A00011AEF0FF00101379191
:101D700036BF3781369F37A111D03651080DF35049
:101D8000396B386F040E3827000E392338C1E9FF4C
:101D9000040E3925EA6E840EEF6E0AD03651080D16
:101DA000F350396BE96E040E3925EA6E840EEF6E3E
:101DB000000122EF0FF00101379136BF3781369FC6
:101DC00037A111D03651080DF3503A6B396F040E1C
:101DD0003927000E3A2339C1E9FF040E3A25EA6E8D
:101DE000EFCF38F10AD03651080DF3503A6BE96E57
:101DF000040E3A25EA6EEFCF38F138AF02D038B58D
:101E000002D0000E01D0010E016E00012EEF0FF086
:101E100014C436F158D701522EE004011151010AC1
:101E2000000105E0020A0BE0030A11E022D014C40D
:101E300036F178D70101396B00019ADC1CD014C44B
:101E400036F194D70101396B000192DC14D0040102
:101E5000506B516B14C436F10001ADD7015203E051
:101E6000010E0401506F020E0101396F000180DC88
:101E700002D081DC00D05CEF0FF00401115100D0E2
:101E8000000179DC00D05CEF0FF01F6A04011051F3
:101E90007F0B000107E0010A07E0030A07E0230ABD
:101EA00007E008D05CD608D0B5D606D0B1D704D0AC
:101EB000E4D702D060DC00D09EEF10F00101365173
:101EC000080DF3503C6BE96E040E3C25EA6EEFCF33
:101ED00038F13751020806E138AD02D0376B02D035
:101EE000010E376F3751030813E1840E386F3651F6
:101EF000080DF3503C6B3B6F040E3B27000E3C2358
:101F00003BC1E9FF040E3C25EA6E840EEF6E07D05C
:101F1000372D03D0C80E386F02D0880E386FD89096
:101F20003635036AF2CF3BF1F29E000165EC00F01A
:101F30000900F5CF03F001013BBFF28E396F03C0FA
:101F40003AF13651080DF3503C6B3B6F010E3B25C7
:101F5000016E000E3C21036E01C0E9FF040E032454
:101F6000EA6E39C1EFFF3AB138813AB3388336515E
:101F7000080DF3503C6BE96E040E3C25EA6E38C147
:101F8000EFFF0001000C036A01013B51700FE96E85
:101F90000F0E0320EA6EEF5212E03B51080DF35092
:101FA0003D6B3C6F040E3C27000E3D233CC1E9FF16
:101FB000040E3D25EA6EEFCF3CF13CAF02D0000E9F
:101FC00001D0010E016E0001000C36C13BF1DBDFD8
:101FD000015264E001013651080DF3503C6B3B6F38
:101FE000040E3B27000E3C23010E3B25016E000E24
:101FF0003C21036E01C0E9FF040E0324EA6E37C1E1
:10200000EFFF3951020817E13651080DF3503C6BD0
:102010003B6F040E3B27000E3C233BC1E9FF040E3F
:102020003C25EA6EEFCF3AF13AAD02D0396B02D0DF
:10203000010E396F13D03951040810E13651080DE3
:10204000F3503C6BE96E040E3C25EA6EEFCF3AF19B
:102050003AAD03D0010E396F01D0396B392D03D061
:10206000C80E3A6F02D0880E3A6F38B13A8138B351
:102070003A833651080DF3503C6B3B6F040E3B27FF
:10208000000E3C233BC1E9FF040E3C25EA6E3AC139
:10209000EFFF010E016E05D000D00001000E016EB1
:1020A00001010001000C0101365304E1000135EC8F
:1020B0000BF001010001000C37C16EFF0101375325
:1020C00003E0040E266E02D0020E266E00016EEFB3
:1020D00010F0206A1F6A28C037F1EED77FEF10F0AA
:1020E000010136530DE11F2C05D00001BEEC0BF0B1
:1020F00006D001011F50020803E10001EAD70101E7
:102100000001000C6C300101346F343334331F0E86
:1021100034176C524EE1040100513C0B0101356F44
:10212000430E04010017000196EC0BF0010135513C
:10213000340822E10401046B0001A7D66D98273C06
:1021400007D00101366B030E376F0001B7DE12D0E6
:102150000101366B020E376F0001B0DE2750FE081A
:1021600009E00101366B386B27C037F1040E396F77
:1021700000012BDF1CD001013551040819E1366B39
:10218000000191DF0101366B020E376F000196DE10
:102190002750FE080CE0273C01D009D00101366B26
:1021A000386B27C037F1010E396F00010EDF0101D6
:1021B0006BD06C5004081DE1430E040104170001AC
:1021C00096EC0BF0FF0E276E0101366B000188DFE5
:1021D000273C01D00AD00101366B386B27C037F19C
:1021E000020E396F0001F1DE02D035EC0BF04BD05E
:1021F00001016CB41FD03451080DF350376B016EE0
:10220000040E3725036E3451080DF350396BE96E17
:10221000040E3925EA6EEF50430B03C0EAFF01C0FC
:10222000E9FFEF6E000196EC0BF034C136F13BDFB5
:102230002AD001013451080DF350376B366F040E6C
:102240003627000E372336C101F0040E3725036E02
:102250003451080DF350396B386F040E3827000ED7
:10226000392338C1E9FF040E3925EA6EEF50430BDC
:1022700003C0EAFF36C1E9FFEF6E000196EC0BF0F8
:1022800034C136F12DDF010100017BEF11F0265240
:1022900001E13AD0685238E068A404D069A402D0C1
:1022A0002DEF0BF06DA201D02FD068AA04D069AA3F
:1022B00002D045EF0BF068A204D069A202D04CEF27
:1022C0000BF068A004D069A002D09BEF0BF068A8C7
:1022D00004D069A802D0B0EF0BF068AC04D069ACB0
:1022E00002D0B5EF0BF00101336B68A606D069A6EA
:1022F00004D0000107D702D0010105D001013351FC
:10230000332B0308F2E20001A19A32EF00F0C9502A
:1023100036C1C9FFC6889E96C7B0FED7016AC6B847
:10232000012AC8EF11F0C7BA04D00101076BC7B486
:10233000078F01010751072B346F34517F0818E3D1
:10234000C69C9EA6FED7C950C688336F342D02D0D6
:1023500033C1F6F0345102080BE1036A0001F65173
:10236000F70FE96E000E0320EA6E33C1EFFF0101A3
:10237000345180080EE1036A0001F651F70FE96E4F
:10238000000E0320EA6EEFCF35F135C136F1BFD72D
:1023900001019E96000132EF00F09EA8FED7AD6EBF
:1023A000000C01010A6B0A51000130EC06F001013A
:1023B0000A2B0001F2DF0C0E01010A5DF4E1F2CFFD
:1023C0000AF1F29EA96AA69CA69EA680A8500ABF02
:1023D000F28E426E42507F0816E3C80E426EA96A22
:1023E000A86EA69CA69EA684F2CF00F0F29E0F01D6
:1023F000550EA76EAA0EA76EA682A6B2FED7A69409
:102400000050F212010100013FEF25F0010EEA6ECB
:102410000B0EE96EEF500EE0070E016E006A002E03
:10242000FED7012EFBD7C70E006E002EFED7000090
:10243000EF2EF2D7000C080E01011A6F1A530FE0AD
:1024400081961951800B02E1819801D0818800D0DA
:1024500000D000D08186D89019371A07EFD7000135
:10246000000C819A819C14C119F1E5DF818C000C6C
:1024700001011251070B4009136F146F0001F1DFC6
:10248000010111517F0B8009136F146F0001E9DF07
:10249000000C818A819C18C119F1CDDF818C000C60
:1024A0000101116B126B0001E3DF010E446EF80EA7
:1024B000436E435202E1445209E00101186B0001EE
:1024C000E8DF4350D8B444064306F3D789EF12F04F
:1024D000818A818C819E0A0E01010B6F000196DFBB
:1024E000818E210E0101146F0001BBDF42C014F187
:1024F000B8DF130E0101146F0001B3DF200E0101DC
:10250000146F0001AEDF090E0101146F0001A9DF95
:10251000C7D7080E0101146F0001A3DF0C0E0101E3
:10252000146F00019EDF000C3F501F0801E33CD0F8
:102530003F507F0801E238D03E6A3E50040830E345
:102540003F504F0813E33F50E00F050DF3CF40F02D
:102550003E504024036AF2CF18F1F29E14EC01F0D1
:10256000010118BFF28E416E15D000013F504F0897
:1025700012E23F50B00F050DF3CF40F03E50402423
:10258000036AF2CF18F1F29E99EC01F0010118BF35
:10259000F28E416E000141C018F17BDF3E2ACDD79B
:1025A0000101186B000175DFD9EF12F017C13FF080
:1025B000BBD7000C01011151016A105D03E210C18B
:1025C00000F00CD0006A080E126F1037003611515F
:1025D000005CD8B0006E0136122FF7D70001000C56
:1025E00001500AC110F1640E0101116F0001E2DF18
:1025F00000C00AF10150300E08E101010BA30ED01A
:102600000BB70CD00BB9200E04D001010B970B991E
:102610000B81012601509EA8FED7AD6E0AC110F1B4
:102620000A0E116F0001C6DF00C00AF10150300E22
:1026300008E101010BB70BD00BA109D00BB9200E9B
:102640000001012601509EA8FED7AD6E0101300E9B
:102650000A270A519EA8FED7AD6E0001BDEF13F008
:102660001E0E0101116F010E126F000101DF4C0EF1
:102670000101176F00019ADF430E0101176F00017E
:1026800095DF440E0101176F000190DF0C0E010170
:10269000116F020E126F0001EBDE01010A6B0A518D
:1026A000000144EC06F001010A2B006E176F0001D7
:1026B0007DDF0A0E01010A5DF2E1180E116F030EB3
:1026C000126F0001D5DE01010A6B0A51000157ECBF
:1026D00006F001010A2B006E176F000167DF060E7E
:1026E00001010A5DF2E1030E116F050E126F000188
:1026F000BFDE01010A6B0A51000168EC06F001011E
:102700000A2B006E176F000151DF0D0E01010A5DEB
:10271000F2E10A6B0A5100017CEC06F001010A2B80
:1027200000013BDE0D0E01010A5DF4E181A429D018
:10273000423C01D026D0010E4226C80E0B6F00018C
:1027400065DE210E0101146F00018BDE42C014F121
:1027500088DE01010A6B0A51000190EC06F00101CC
:102760000A2B00011ADE050E01010A5DF4E142C0E8
:102770000AF11B0E0B6F000133D7200E0EDE010194
:10278000D5D7423C03D0800E426EC3D7A96A42C05F
:10279000A8FFA69CA69EA684F2CF00F0F29E0F0191
:1027A000550EA76EAA0EA76EA682A6B2FED7A69455
:1027B0000050F21200018CDE43EF25F06D6A696A69
:1027C000080E6F6E945030090101946E266A186AE3
:1027D000F2BE188EF29E000182EC0BF018BEF28E53
:1027E000F3EF13F0EBD718EF14F0186AF2BE188E5F
:1027F000F29E82EC0BF018BEF28E6D6A140E6F6EB4
:10280000696A6D86010E266E09EF14F06DB601D06F
:10281000ECD7262C0BD06DBA09D0686A696AA08AF9
:10282000C00EF212110E696E020E266E000CDAD77F
:10283000EDDF26500208FCE145EF25F0EACF12F16A
:10284000E9CF11F101010B39F0090D6F0D27E20FEE
:102850000E6F320F106F0B510F0B0E270E27102724
:10286000E90F0F6F0F270F270A390F0B0F271027BC
:102870000F371037101F10370A510F0B10270D3765
:10288000070E0C6F0A0E0F071027FDE30E070F2728
:10289000FDE30D070E27FDE30C070D27FDE3010EF9
:1028A000EA6E0C0EE96E070E1115119DE926100E49
:1028B000E95CD8B4118DEF50006E08E111BD06D06F
:1028C00011B90CD011B702D0200E03D01187119985
:1028D000300E002600509EA8FED7AD6EEE5011AD12
:1028E000E6D70001000C8E0E006E0BC101F00AC18C
:1028F00002F0036A015209E102C001F0026A080E07
:10290000005E015202E1006A08D0D89001BE04D0F6
:10291000023601360006F9D7019E57EF27F0010174
:102920002351D8B471D0006E2751D8B46DD0002691
:1029300004E3810E002668E204D07F0E005E64E3AB
:1029400063E024C12BF128512B1B248F288F2651A3
:102950002A03F4CF2DF125512903F4CF03F0F3CF4F
:102960002CF12A03F3502D27F4502C23000E0322C0
:1029700026512903F3502D27F4502C23000E026A10
:102980000322022224512A03F3502C27F45003225D
:10299000000E022224512903F3500326F450022290
:1029A000000E016A012226512803F3502C27F4500F
:1029B0000322000E0222012225512803F350032690
:1029C000F4500222000E012224512803F350022663
:1029D000F4500122002A01BE05D02C3703360236FE
:1029E00001360006000E2CAF0AD0032A0222012273
:1029F000015005E1025003E1035001E1002A2BBF21
:102A0000018E2BAF019E04D0006A016A026A036A3C
:102A10000001000C800ED8A202D00101281B010188
:102A20002D6B2E6B24C12CF128512C1B2351D8B4B3
:102A3000DFD02B6F006E2751D8B4E3D02B5FD8B412
:102A400083D03EE328C131F1318F29C130F12AC151
:102A50002FF12E6BD890313330332F332E332B2F71
:102A6000F8D72CAF03D02D81E0D02D912B912D895B
:102A7000010EEA6E260EE96EEBD02D992CBF0AD01E
:102A80002BA113D0313330332F332E33002AD8B457
:102A9000C7D00BD031BF0CD0D8902E372F3730375E
:102AA00031370006D8B4BCD0F5D72D8D6DD02D9D13
:102AB00024C12CF124AF02D0318FABD0319FA9D0EB
:102AC00027C12BF127C100F023512B5F24C131F125
:102AD000318F25C130F126C12FF12E6BD8903133C3
:102AE00030332F332E332B2FF8D72CAF03D02D8339
:102AF0009CD02D932B912D8B010EEA6E2A0EE96E40
:102B0000A7D02D9B2CBF0AD02BA113D0313330334B
:102B10002F332E33002AD8B483D00BD031BF0CD042
:102B2000D8902E372F37303731370006D8B478D0C9
:102B3000F5D72D8F29D02D9F28C12CF128AF02D099
:102B4000318F67D0319F65D028C131F1318F29C1D4
:102B500030F12AC12FF12CAF04D0319F2D8565D0E3
:102B60002D952E6B2B91010EEA6E260EE96E70D01C
:102B70002CBF1CD024C12CF12BA106D03133303313
:102B80002F332E33002A4CE02EAF0BD02F2B09E130
:102B9000302B07E1312B05E1313330332F33002A5D
:102BA0003FE02DBD84D72DBFC6D71CD0800E311B72
:102BB00031AF04D03AD028C12CF10AD024C12CF175
:102BC000315306E1305304E12F5302E1006A21D072
:102BD00031BF08D0D8902E372F3730373137002EFD
:102BE000F7D71ED02CAF02D0318F13D0319F11D028
:102BF00027C100F028C131F129C130F12AC12FF1DC
:102C000008D023C100F024C131F125C130F126C123
:102C10002FF131C101F030C102F02FC103F034D0E7
:102C2000006A016A026A036A2FD02E6B2F1F301FC1
:102C3000311F2E1F2E2B05E12F2B03E1302B01E13D
:102C4000312B2DB112D72DB354D72DB589D7B3D78A
:102C5000EF502F2705E3302B03E1312BD8B42B8124
:102C6000ED52EF50302703E3312BD8B42B81ED52D6
:102C7000EF50EFBE01D0800A3127D8B02B812DB99B
:102C8000FCD62DBB3ED774D70001000C0101116B9F
:102C90000AC112F1000138EC12F001010B6B0B516B
:102CA0000001A2EC06F001010B2B006E176F000172
:102CB0007DDC0E0E01010B5DF2E10001F7EF27F064
:102CC00001011751B608176F036A18C11BF1188F5D
:102CD000D890183319331A330332023201320032DA
:102CE000172FF6D71BAF0BD0001E011E021E031EAE
:102CF000002AD8B4012AD8B4022AD8B4032A000181
:102D0000000C006A016A026A036A01011F6B206BF2
:102D1000216B226B1E511D111C111B112CE0200E6A
:102D2000236FD8901737183719371A371F372037BE
:102D3000213722371E51225D08E11D51215D05E139
:102D40001C51205D02E11B511F5D0FE31B511F5FF2
:102D50001C51D8A01C3D205F1D51D8A01D3D215FF6
:102D60001E51D8A01E3D225FD880003601360236A3
:102D70000336232FD6D7010EEA6E1F0EE96E00012F
:102D8000000CE95001010F6F0E51116F1BE00DC1D6
:102D900026F10CC125F10BC124F10AC123F12A6BE4
:102DA000296B200E286F820E276F0001B8DD03C04B
:102DB0000DF102C00CF101C00BF100C00AF10101DC
:102DC000112FE5D70DC11AF10CC119F10BC118F182
:102DD0000AC117F1000174DF03C00DF102C00CF14C
:102DE00001C00BF100C00AF101010DAF0DD00F07BA
:102DF0000F8B0A1F0B1F0C1F0D1F0A2BD8B40B2B98
:102E0000D8B40C2BD8B40D2B3B0E166F9A0E156F41
:102E1000CA0E146F136B0A0E116F0E51D8B40F2B1C
:102E20000DC11AF10CC119F10BC118F10AC117F14A
:102E300016C11EF115C11DF114C11CF113C11BF106
:102E400000015FDF0150EFCF0AF1ECCF0BF1ECCFC7
:102E50000CF1ECCF0DF1005213E101010E29115DCF
:102E6000D8A402D000010CD00F510DE00F0B115D62
:102E700001E03CE20FBF3AD00FBD05D0200E31D0AB
:102E8000200E01010F170FAB0DD00F9B0E51D8A4D0
:102E90000F0700500F6F2D0E9EA8FED7AD6E0F517D
:102EA000006E0F6B0E51115D0BE100500F6F2E0E77
:102EB0009EA8FED7AD6E0F51006E200E0F17000EAC
:102EC000300E0FAB0ED00F9B0E51D8A40F07005041
:102ED0000F6F2D0E9EA8FED7AD6E0F51006E0F6BBB
:102EE000300E002600509EA8FED7AD6E16C11AF116
:102EF00015C119F114C118F113C117F11E6B1D6B27
:102F00001C6B0A0E1B6F0001FCDE03C016F102C031
:102F100015F101C014F100C013F10101112F80D788
:102F20000001000CE95001010F6F0E51116F1BE001
:102F30000DC126F10CC125F10BC124F10AC123F109
:102F40002A6B296B200E286F820E276F0001E7DCA9
:102F500003C00DF102C00CF101C00BF100C00AF179
:102F60000101112FE5D77E0E006E016A0BBF018EA5
:102F7000026A036AD8920DC126F10CC125F10BC17A
:102F800024F10AC123F103C02AF102C029F101C0D2
:102F900028F1276F00013EDD03C00DF102C00CF1E6
:102FA00001C00BF100C00AF10DC11AF10CC119F1F9
:102FB0000BC118F10AC117F183DE03C00DF102C085
:102FC0000CF101C00BF100C00AF101010DAF0DD0F1
:102FD0000F070F8B0A1F0B1F0C1F0D1F0A2BD8B4D6
:102FE0000B2BD8B40C2BD8B40D2B3B0E166F9A0EAE
:102FF000156FCA0E146F136B0A0E116F0E51D8B4F1
:103000000F2B0DC11AF10CC119F10BC118F10AC136
:1030100017F116C11EF115C11DF114C11CF113C128
:103020001BF100016EDE0150EFCF0AF1ECCF0BF186
:10303000ECCF0CF1ECCF0DF1005213E101010E29A0
:10304000115DD8A402D000010CD00F510DE00F0B80
:10305000115D01E044E20FBF42D00FBD05D0200E4C
:1030600037D0200E01010F170FAB0FD00F9B0E5161
:10307000D8A40F0700500F6F2D0E176F0001D6EC6C
:1030800012F001010F51006E0F6B0E51115D0DE139
:1030900000500F6F2E0E176F0001D6EC12F00101D9
:1030A0000F51006E200E0F17000E300E0FAB10D018
:1030B0000F9B0E51D8A40F0700500F6F2D0E176FE6
:1030C0000001D6EC12F001010F51006E0F6B300EB3
:1030D000002600C017F10001D6EC12F0010116C164
:1030E0001AF115C119F114C118F113C117F11E6BB2
:1030F0001D6B1C6B0A0E1B6F000103DE03C016F173
:1031000002C015F101C014F100C013F10101112F2B
:1031100078D70001000C0101186B000149EC12F096
:10312000060E0101186F000149EC12F0090E0101B1
:10313000186F000149EC12F0090E0101186F00012F
:1031400049EC12F0060E0101186F000149EC12F073
:103150000101186B000149EC12F0000C030E010193
:103160000B5F0BE3010EEA6E0B0EE96EEF5005E00C
:1031700002D000D00000EF2EFCD70001000C016A45
:10318000026A006A036A01010F5102E10E5118E060
:10319000100E106FD8900C370D37003603360F51D4
:1031A000035C02E10E51005C07E30E51005ED8A003
:1031B00003060F51035ED88001360236102FEAD77E
:1031C0000001000C01010C510E03F3CF01F0F4CF0C
:1031D00000F00F03F35000260D510E03F3500020B2
:1031E000026E0001000CEACF12F1E9CF11F10101EA
:1031F0000BAF08D0118F11A9112B0A1F0B1F0A2B1F
:10320000D8B40B2B0B39F0090D6F0D27E20F0E6FA1
:10321000320F106F0B510F0B0E270E271027E90FDF
:103220000F6F0F270F270A390F0B0F2710270F37A4
:103230001037101F10370A510F0B10270D37070ECC
:103240000C6F0A0E0F071027FDE30E070F27FDE393
:103250000D070E27FDE30C070D27FDE3010EEA6EB7
:103260000C0EE96E070E1115119DE906111507E107
:1032700011B9E92A11B903D0200E006E1CD0E9263D
:10328000100EE95CD8B4118DEF50006E08E111BD4D
:1032900006D011B914D011B702D0200E0BD011AF47
:1032A00006D02D0E006EED50119D119F04D0118798
:1032B0001199300E002600509EA8FED7AD6EEE503C
:1032C00011ADDED70001000C8E0E006E12C101F0B0
:1032D00011C102F0036A01AE05D0011E021E022ACE
:1032E00001E1012A015209E102C001F0026A080E5F
:1032F000005E015202E1006A0DD0D89001BE04D0F8
:10330000023601360006F9D7010112AF02D00001E2
:1033100001D0019E0001000C01012351D8B4A5D0B9
:103320002F6F2751D8B4A1D02F5F05E37F0E2F2731
:10333000D8B09BD006D0810E2F5FD8A096D0D8B43D
:1033400094D02FC100F0016A026A036A2E6B24C177
:103350002DF12D8F25C12CF126C12BF1190E2F6FC8
:103360002A512B5F0DE2010E2C5F0AE22D5F08E26D
:103370002E5F06E22E2B2D2B2C2B2A512B2728D00B
:1033800029512C5F12E2010E2D5F0FE22E5F0DE23C
:103390002E2B2D2B29512C272A512B2719E32C2B8F
:1033A00017E12D2B15E12E2B13D0285180092D5F0D
:1033B0000EE2010E2E5F0BE22E2B285180092D27E5
:1033C00029512C27E9E32D2BE7E12E2BE5D70380AC
:1033D0002F2F01D00BD0D8902B372C372D372E37ED
:1033E000D8900336023601363037BAD730A106D02E
:1033F000D890013202320332303302D0000635E079
:1034000030BF1ED0D8902B372C372D372E372A516E
:103410002B5F07E2010E2C5F04E22D5F02E22E5FBC
:103420001AE329512C5F05E2010E2D5F02E22E5FA7
:1034300012E3285180092D5F03E2010E2E5F0BE39A
:10344000032A09E1022A07E1012A05E1002A0DE029
:1034500001320232033224C12FF128512F1B2FAF2A
:1034600002D0018E06D0019E04D0006A016A026A71
:10347000036A0001000C20C127F101012451271B20
:1034800027AF05D0D894D89020BFD8802FD020C1A6
:1034900027F123C128F11F51285F06E027AF26D06E
:1034A000D850010AD86E22D024C128F12051285FBB
:1034B00006E027AF1BD0D850010AD86E17D025C11F
:1034C00028F12151285F06E027AF10D0D850010A1B
:1034D000D86E0CD026C128F12251285F06E027AF14
:1034E00005D0D850010AD86E01D0D8900001000C48
:1034F00001011E911E9311C115F110C114F10FC1EC
:1035000013F10EC112F111C122F110C121F10FC14D
:1035100020F10EC11FF1266B256B246B236B00017C
:10352000AADF05E301011E811351800A136F010117
:10353000226B216B206B7F0E1F6F15C126F114C10A
:1035400025F113C124F112C123F1000194DF1AE324
:103550000101266B256B246B7F0E236F15C12AF1A9
:1035600014C129F113C128F112C127F10001D4DEE1
:1035700003C015F102C014F101C013F100C012F133
:1035800001011E830A0E0101266F890E256F340E7C
:10359000246F7C0E236F15C12AF114C129F113C1C8
:1035A00028F112C127F100018FEC14F000C01FF1C7
:1035B00001C020F102C021F103C022F103C026F1B5
:1035C00002C025F101C024F100C023F115C12AF188
:1035D00014C129F113C128F112C127F18FEC14F0A5
:1035E00000C01FF101C020F102C021F103C022F18F
:1035F000D89203C026F102C025F101C024F100C019
:1036000023F17C0E01012A6F790E296F350E286F88
:10361000810E276F00010AEC15F003C019F102C0FA
:1036200018F101C017F100C016F119C126F118C137
:1036300025F117C124F116C123F115C12AF114C1D6
:1036400029F113C128F112C127F18FEC14F000C049
:103650001FF101C020F102C021F103C022F103C01B
:1036600026F102C025F101C024F100C023F115C1EB
:103670002AF114C129F113C128F112C127F18FECED
:1036800014F000C01FF101C020F102C021F103C0FD
:1036900022F1D89203C026F102C025F101C024F125
:1036A00000C023F13F0E01012A6F020E296F330E75
:1036B000286F830E276F00010AEC15F003C019F183
:1036C00002C018F101C017F100C016F119C126F1AE
:1036D00018C125F117C124F116C123F115C12AF132
:1036E00014C129F113C128F112C127F18FEC14F094
:1036F00000C01FF101C020F102C021F103C022F17E
:1037000003C026F102C025F101C024F100C023F15D
:1037100015C12AF114C129F113C128F112C127F1F1
:103720008FEC14F000C01FF101C020F102C021F1A4
:1037300003C022F1D89203C026F102C025F101C0D6
:1037400024F100C023F1330E01012A6F8C0E296F82
:103750001E0E286F830E276F00010AEC15F003C0C0
:1037600019F102C018F101C017F100C016F10101F2
:10377000266B256B246B7F0E236F15C12AF114C1B4
:1037800029F113C128F112C127F100018FEC14F0C7
:1037900000C01FF101C020F102C021F103C022F1DD
:1037A00003C026F102C025F101C024F100C023F1BD
:1037B00015C12AF114C129F113C128F112C127F151
:1037C0008FEC14F000C01FF101C020F102C021F104
:1037D00003C022F1D89203C026F102C025F101C036
:1037E00024F100C023F11B0E01012A6FE40E296FA2
:1037F000350E286F820E276F00010AEC15F003C00A
:103800001DF102C01CF101C01BF100C01AF11DC165
:1038100026F11CC125F11BC124F11AC123F115C1E8
:103820002AF114C129F113C128F112C127F18FEC3B
:1038300014F000C01FF101C020F102C021F103C04B
:1038400022F103C026F102C025F101C024F100C01D
:1038500023F115C12AF114C129F113C128F112C1B4
:1038600027F18FEC14F000C01FF101C020F102C05D
:1038700021F103C022F1D89203C026F102C025F144
:1038800001C024F100C023F1A40E01012A6FDB0E58
:10389000296F670E286F830E276F00010AEC15F061
:1038A00003C01DF102C01CF101C01BF100C01AF1E0
:1038B0001DC126F11CC125F11BC124F11AC123F140
:1038C00015C12AF114C129F113C128F112C127F140
:1038D0008FEC14F000C01FF101C020F102C021F1F3
:1038E00003C022F103C026F102C025F101C024F17A
:1038F00000C023F115C12AF114C129F113C128F127
:1039000012C127F18FEC14F000C01FF101C020F1AB
:1039100002C021F103C022F1D89203C026F102C0F7
:1039200025F101C024F100C023F1330E01012A6FFB
:103930008C0E296F1E0E286F830E276F00010AEC74
:1039400015F003C01DF102C01CF101C01BF100C045
:103950001AF115C126F114C125F113C124F112C1C8
:1039600023F119C12AF118C129F117C128F116C193
:1039700027F18FEC14F000C01FF101C020F102C04C
:1039800021F103C022F103C026F102C025F101C0DC
:1039900024F100C023F11DC12AF11CC129F11BC172
:1039A00028F11AC127F1B8DC03C019F102C018F1DF
:1039B00001C017F100C016F101011EA31DD0D8826D
:1039C000DB0E266F0F0E256F490E246F7F0E236FBF
:1039D00019C12AF118C129F117C128F116C127F11F
:1039E00000010AEC15F003C019F102C018F101C082
:1039F00017F100C016F101011EA103D01751800A72
:103A0000176F16C100F017C101F018C102F019C1FB
:103A100003F00001000CE95001010F6F0E51116F0E
:103A20001CE00DC126F10CC125F10BC124F10AC126
:103A300023F12A6B296B200E286F820E276F00015D
:103A40008FEC14F003C00DF102C00CF101C00BF1BA
:103A500000C00AF10101112FE4D70DC11AF10CC108
:103A600019F10BC118F10AC117F1000160EC16F051
:103A700003C00DF102C00CF101C00BF100C00AF14E
:103A800001010DAF0DD00F070F8B0A1F0B1F0C1F6D
:103A90000D1F0A2BD8B40B2BD8B40C2BD8B40D2B7C
:103AA0003B0E166F9A0E156FCA0E146F136B0A0E2B
:103AB000116F0E51D8B40F2B0DC11AF10CC119F1B1
:103AC0000BC118F10AC117F116C11EF115C11DF184
:103AD00014C11CF113C11BF1000181EC16F001505F
:103AE000EFCF0AF1ECCF0BF1ECCF0CF1ECCF0DF1F5
:103AF000005213E101010E29115DD8A402D000018A
:103B00000CD00F510DE00F0B115D01E044E20FBF2F
:103B100042D00FBD05D0200E37D0200E01010F1767
:103B20000FAB0FD00F9B0E51D8A40F0700500F6F93
:103B30002D0E176F0001D6EC12F001010F51006E2F
:103B40000F6B0E51115D0DE100500F6F2E0E176FB0
:103B50000001D6EC12F001010F51006E200E0F177C
:103B6000000E300E0FAB10D00F9B0E51D8A40F07D4
:103B700000500F6F2D0E176F0001D6EC12F00101EF
:103B80000F51006E0F6B300E002600C017F10001C0
:103B9000D6EC12F0010116C11AF115C119F114C1C8
:103BA00018F113C117F11E6B1D6B1C6B0A0E1B6FF6
:103BB000000181EC16F003C016F102C015F101C03E
:103BC00014F100C013F10101112F76D700010FEF9E
:103BD0002FF0180E0101116F126B000138EC12F07A
:103BE0003E6A3E505908D8A02CD101010A2D0DD0B3
:103BF000036A3E50F2CF0BF1F29E00011EEC02F080
:103C000001010BBFF28E416EFFD00A5102080DE197
:103C1000036A3E50F2CF0BF1F29E000158EC02F025
:103C200001010BBFF28E416EEFD00A5103080DE186
:103C3000036A3E50F2CF0BF1F29E000192EC02F0CB
:103C400001010BBFF28E416EDFD00A5104080DE175
:103C5000036A3E50F2CF0BF1F29E0001CCEC02F071
:103C600001010BBFF28E416ECFD00A5105080DE164
:103C7000036A3E50F2CF0BF1F29E000106EC03F016
:103C800001010BBFF28E416EBFD00A5106080DE153
:103C9000036A3E50F2CF0BF1F29E000140EC03F0BC
:103CA00001010BBFF28E416EAFD00A5107080DE142
:103CB000036A3E50F2CF0BF1F29E00017AEC03F062
:103CC00001010BBFF28E416E9FD00A5108080DE131
:103CD000036A3E50F2CF0BF1F29E0001B4EC03F008
:103CE00001010BBFF28E416E8FD00A5109080DE120
:103CF000036A3E50F2CF0BF1F29E0001EEEC03F0AE
:103D000001010BBFF28E416E7FD00A510A080DE10E
:103D1000036A3E50F2CF0BF1F29E000128EC04F052
:103D200001010BBFF28E416E6FD00A510B080DE1FD
:103D3000036A3E50F2CF0BF1F29E000162EC04F0F8
:103D400001010BBFF28E416E5FD00A510C080DE1EC
:103D5000036A3E50F2CF0BF1F29E00019CEC04F09E
:103D600001010BBFF28E416E4FD00A510D080DE1DB
:103D7000036A3E50F2CF0BF1F29E0001D6EC04F044
:103D800001010BBFF28E416E3FD00A510E080DE1CA
:103D9000036A3E50F2CF0BF1F29E000110EC05F0E9
:103DA00001010BBFF28E416E2FD00A510F080DE1B9
:103DB000036A3E50F2CF0BF1F29E00014AEC05F08F
:103DC00001010BBFF28E416E1FD00A5110080DE1A8
:103DD000036A3E50F2CF0BF1F29E000184EC05F035
:103DE00001010BBFF28E416E0FD00A5111080CE198
:103DF000036A3E50F2CF0BF1F29E0001BEEC05F0DB
:103E000001010BBFF28E416E3E501E0809E1180EF3
:103E1000116F010E126F000138EC12F00BD001018E
:103E20003E503C0807E1180E116F020E126F0001A0
:103E300038EC12F041C018F1000149EC12F03E2AB2
:103E4000D0D6000C150E0101116F040E126F000187
:103E500038EC12F03E6A3E50230812E3036A3E50EB
:103E6000F2CF0AF1F29EF8EC05F001010ABFF28EE2
:103E7000416E41C018F1000149EC12F03E2AEBD727
:103E8000AFEF32F00101116B126B000138EC12F050
:103E90003E6A3E50170831E3036A3E50F2CF0AF102
:103EA000F29E17EC06F001010ABFF28E416E3E5001
:103EB000060808E1116B010E126F000138EC12F0D8
:103EC00015D001013E500C0808E1116B020E126F73
:103ED000000138EC12F00AD001013E50120806E150
:103EE000116B030E126F000138EC12F041C018F193
:103EF000000149EC12F03E2ACCD7B1EF32F08E0E21
:103F0000006E01011151005E12C102F013C101F0F7
:103F1000028E005209E0D890025202E1015204E000
:103F200002320132002EF7D712AF05D0011E021E59
:103F3000012AD8B4022A0001000C200E01010BA9AD
:103F4000300E0C6F0AC100F00AAF07D0001E002A25
:103F500000C00AF12D0E0C6F0B8F01500AC110F139
:103F6000640E116F0001DAEC12F000C00AF1300E9D
:103F7000012401010D6F0AC110F10A0E116F000139
:103F8000DAEC12F0300E002401010F6F300E012424
:103F90000E6F0CC100F00BA702D00BAF0B950BB945
:103FA0000BD00BAF22D00BB520D000C00DF10BB35E
:103FB0001CD000C00EF119D0300E0D5D16E100C00E
:103FC0000DF1200E0C6F0BA704D00B950B830BAFDC
:103FD0000B93300E0E5D09E100C00EF1200E0D6F47
:103FE0000BA7F7D70B930BAF0B910BA506D00CC10A
:103FF00017F10001D6EC12F001010BA306D00DC1A0
:1040000017F10001D6EC12F001010BA105D00EC191
:1040100017F10001D6EC12F00FC117F10001D6EC38
:1040200012F0000C200E01010BA9300E0C6F0AC11A
:1040300000F00AAF07D0001E002A00C00AF12D0EC2
:104040000C6F0B8F01500AC110F1640E116F00014B
:10405000DAEC12F000C00AF1300E012401010D6FFC
:104060000AC110F10A0E116F0001DAEC12F0300EE5
:10407000002401010F6F300E01240E6F0CC100F0FF
:104080000BA702D00BAF0B950BB90BD00BAF22D007
:104090000BB520D000C00DF10BB31CD000C00EF149
:1040A00019D0300E0D5D16E100C00DF1200E0C6F21
:1040B0000BA704D00B950B830BAF0B93300E0E5D4B
:1040C00009E100C00EF1200E0D6F0BA7F7D70B937F
:1040D0000BAF0B910BA504D00C519EA8FED7AD6E73
:1040E0000BA304D00D519EA8FED7AD6E0BA104D03A
:1040F0000E519EA8FED7AD6E0F519EA8FED7AD6E95
:104100000001000C818A819C080E0101126F12537C
:1041100011E08196030E006E002EFED700D01151E3
:10412000010B02E1819801D081888186D8901133FA
:104130001207EDD7818C0001000C0101126B0AC13E
:1041400011F111BF1207000164EC19F003C010F166
:1041500002C00FF101C00EF100C00DF110C122F13B
:104160000FC121F10EC120F10DC11FF10101266B1C
:10417000256BB60E246F850E236F00013BEC1AF001
:1041800001E208E10101106B0F6BB40E0E6F850E9A
:104190000D6F1BD00101226B216B360E206F850E37
:1041A0001F6F10C126F10FC125F10EC124F10DC101
:1041B00023F100013BEC1AF001E207E10101106B71
:1041C0000F6B340E0E6F850E0D6F080E0101116F0F
:1041D000126B000138EC12F0200E0101176F000184
:1041E000D6EC12F0080E0101116F010E126F0001E2
:1041F00038EC12F0200E0101176F0001D6EC12F01E
:10420000080E0101116F020E126F000138EC12F05E
:10421000200E0101176F0001D6EC12F0080E01010B
:10422000116F030E126F000138EC12F0200E010125
:10423000176F0001D6EC12F00101226B216B400ECA
:10424000206F800E1F6F10C126F10FC125F10EC126
:1042500024F10DC123F100013BEC1AF030E310C151
:1042600026F10FC125F10EC124F10DC123F1010189
:104270002A6B296B340E286F810E276F00018CEC9E
:1042800019F0D8820101266B256B246B830E236FF6
:1042900003C02AF102C029F101C028F100C027F1B2
:1042A00000010AEC15F003C014F102C013F101C0C3
:1042B00012F100C011F123DE01C00CF17AD010C15F
:1042C00022F10FC121F10EC120F10DC11FF1010139
:1042D000266B256BC00E246F800E236F00013BEC14
:1042E0001AF041E30DC111F101010E51800A126F64
:1042F0000FC113F110C114F110C126F10FC125F146
:10430000246F0DC123F12A6B296B340E286F810EA7
:10431000276F00018CEC19F000C011F101C012F1FF
:1043200002C013F103C014F1D89203C026F102C0F9
:1043300025F101C024F100C023F101012A6B296B92
:10434000700E286F820E276F00010AEC15F003C073
:1043500014F102C013F101C012F100C011F1CFDD60
:1043600001C00CF126D0080E01010B6F0B510E0895
:104370001EE00BC111F1020E126F000138EC12F0B9
:10438000010E0101186F000149EC12F00BC111F18F
:10439000010E0101126F000138EC12F0800E0101D4
:1043A000186F000149EC12F001010B2BDFD758D038
:1043B0000001496A486A476A466A468001010B6BF8
:1043C0000C510B5D07E0D8904636473648364936E3
:1043D0000B2BF6D746C056F0576A586A596A47C041
:1043E00052F0536A546A556A48C04EF04F6A506A98
:1043F000516A49C04AF04B6A4C6A4D6A080E0B6F0D
:104400000B510E082DE00BC111F1126B000138ECBD
:1044100012F04AC011F176DE0BC111F1010E01015B
:10442000126F000138EC12F04EC011F16BDE0BC1BF
:1044300011F1020E0101126F000138EC12F052C0AE
:1044400011F160DE0BC111F1030E0101126F0001C9
:1044500038EC12F056C011F155DE01010B2BD0D70C
:104460000001A6EF33F00101126B0AC111F111BF77
:104470001207000164EC19F003C00FF102C00EF145
:1044800001C00DF100C00CF10FC122F10EC121F1EC
:104490000DC120F10CC11FF10101266B256BB60E79
:1044A000246F850E236F00013BEC1AF001E208E156
:1044B00001010F6B0E6BB40E0D6F850E0C6F1BD0D0
:1044C0000101226B216B360E206F850E1F6F0FC10D
:1044D00026F10EC125F10DC124F10CC123F100011B
:1044E0003BEC1AF001E207E101010F6B0E6B340E99
:1044F0000D6F850E0C6F150E0101116F030E126FFB
:10450000000138EC12F00101106B10510001B7EC02
:1045100006F00101102B006E176F0001D6EC12F0AF
:10452000060E0101105DF1E1226B216B400E206F40
:10453000800E1F6F0FC126F10EC125F10DC124F1B0
:104540000CC123F100013BEC1AF045E30FC126F149
:104550000EC125F10DC124F10CC123F101012A6B1B
:10456000296B200E286F810E276F00018CEC19F04B
:10457000D8820101266B256B1C0E246F840E236FDD
:1045800003C02AF102C029F101C028F100C027F1BF
:1045900000010AEC15F003C014F102C013F101C0D0
:1045A00012F100C011F1ABDC01C00BF10BC111F134
:1045B000030E0101126F000138EC12F07E0E0101B2
:1045C000186F000149EC12F0200E0101176F000175
:1045D000D6EC12F08AD00FC122F10EC121F10DC12B
:1045E00020F10CC11FF10101266B256BC00E246F59
:1045F000800E236F00013BEC1AF055E30CC110F163
:1046000001010D51800A116F0EC112F10FC113F19A
:104610000FC126F10EC125F1246F0CC123F12A6BC5
:10462000296B200E286F810E276F00018CEC19F08A
:1046300000C010F101C011F102C012F103C013F16A
:10464000D89203C026F102C025F101C024F100C0B8
:1046500023F101012A6B296B180E286F840E276F36
:1046600000010AEC15F003C014F102C013F101C0FF
:1046700012F100C011F143DC01C00BF10BC111F1CB
:10468000030E0101126F000138EC12F07E0E0101E1
:10469000186F000149EC12F0200E0101176F0001A4
:1046A000D6EC12F022D0260E0101116F030E126F0C
:1046B000000138EC12F07E0E0101186F000149EC88
:1046C00012F0270E0101116F030E126F000138EC7A
:1046D00012F07E0E0101186F000149EC12F0200E5D
:1046E0000101176F0001D6EC12F0AAEF33F0205051
:1046F000016E000C010E01010A6F0001F8DF01C01C
:104700000BF101010A5310E008530EE10C6B0C5140
:1047100000019DEC0AF001010C2B0001CDEC11F021
:104720002C0E01010C5DF3E10A5310E108530EE079
:104730000C6B0C510001C1EC0AF001010C2B0001C3
:10474000CDEC11F02E0E01010C5DF3E10B5310E0E6
:1047500009530EE10C6B0C510001E6EC0AF001016B
:104760000C2B0001CDEC11F01C0E01010C5DF3E1EE
:104770000B5310E109530EE00C6B0C51000102ECDD
:104780000BF001010C2B0001CDEC11F03A0E0101F0
:104790000C5DF3E10AC108F10BC109F10001000C45
:1047A000186AF2BE188EF29E0AC13BF1C3EC0FF0FC
:1047B00018BEF28E015248E001010A51080DF35073
:1047C000136B126F040E1227000E1323020E122514
:1047D000016E000E1321036E01C0E9FF040E0324D5
:1047E000EA6EECCF03F0ED52EFCF10F103C011F100
:1047F00011C1EAFF10C1E9FF0CC1E2FF0BC1E1FFEB
:104800000EC102F00DC101F0015202E0022A02D0F5
:10481000025206E0E6CFEEFF012EFCD7022EFAD7B9
:10482000186AF2BE188EF29E0AC136F10EC138F136
:104830000DC137F10FC139F10001E5EC0FF018BEE1
:10484000F28E015003D000D0000E016E000C036AFE
:1048500001010A51700FE96E0F0E0320EA6EEF524C
:104860000DE00A51080DF3500C6B0B6FE96E040E4E
:104870000C25EA6EEFCF0BF10BAF02D0000E01D08A
:10488000010E016E00013FEF34F001010F51080DE0
:10489000F3501A6B196F020E1925016E000E1A21C2
:1048A000036E01C0E9FF040E0324EA6EECCF03F0AF
:1048B000ED52EFCF14F103C015F10F51080DF35075
:1048C0001A6B196F010E1925016E000E1A21036E65
:1048D00001C0E9FF040E0324EA6EEF50036A176F6C
:1048E00003C018F10F51080DF3501A6BE96E040E56
:1048F0001A25EA6EEFCF16F116B1188116B3188398
:104900001851135D08E303E11251175D04E218C169
:1049100013F117C112F111C1EAFF10C1E9FF15C16E
:10492000E2FF14C1E1FF13C102F012C101F0015214
:1049300002E0022A02D0025206E0E6CFEEFF012E8C
:10494000FCD7022EFAD712C101F013C102F0000108
:10495000B5EF24F00AC10FF10CC111F10BC110F138
:104960000EC113F10DC112F190D702C00EF101C0BA
:104970000DF1186AF2BE188EF29E0AC136F1020ECF
:104980000101376F00015EEC0FF018BEF28E0101DD
:104990000DC101F00EC102F000014DEF34F0010134
:1049A0000BBF10D00F0E006E0A3900160A0E005C05
:1049B00003E2300E002602D00B51002600509EA8C4
:1049C000FED7AD6E0F0E0A170A0E0A5D02E2300E18
:1049D00002D00B9F0B510A270A519EA8FED7AD6E3D
:1049E0000001000CF86AD09E088EFE0E006E040EC8
:1049F000016E020EE96E000EEA6EEE6A002EFDD721
:104A0000012EFBD7600E006E040E016EA00EE96E43
:104A1000040EEA6EEE6A002EFDD7012EFBD7EA6A7D
:104A2000E96A93829380A00EC86E360EC66EB89661
:104A30000C0EAF6EA60EAC6E900EAB6EC150C00BDE
:104A40000F09C16E070EB46E196A1A6A236A040E42
:104A5000246E0C0E256E266A2A6A766B030E0101FF
:104A6000076FC00EF2129D862F0E926E070E936E88
:104A7000950E946E929889980001D1EF11F068EC30
:104A800012F030EF13F017EF14F0786B020E776F1F
:104A9000F2CF0AF1F29E010EA96EA69CA69EA680F8
:104AA000A85001010ABFF28E0001D06FF2CF0AF1C7
:104AB000F29E020EA96EA69CA69EA680A850010199
:104AC0000ABFF28E0001CF6FF2CF0AF1F29E200EE4
:104AD000A96EA69CA69EA680A85001010ABFF28ED0
:104AE0000001B26BB16FB1C0B2F0B16BF2CF0AF19D
:104AF000F29E100EA96EA69CA69EA680A85001014B
:104B00000ABFF28E0001B127000EB223F2CF0AF1E4
:104B1000F29E210EA96EA69CA69EA680A850010119
:104B20000ABFF28E0001B46BB36FB3C0B4F0B36BC5
:104B3000F2CF0AF1F29E110EA96EA69CA69EA68047
:104B4000A85001010ABFF28E0001B327000EB42362
:104B5000F2CF0AF1F29E220EA96EA69CA69EA68016
:104B6000A85001010ABFF28E0001B66BB56FB5C047
:104B7000B6F0B56BF2CF0AF1F29E120EA96EA69CAA
:104B8000A69EA680A85001010ABFF28E0001B5279B
:104B9000000EB623F2CF0AF1F29E230EA96EA69C58
:104BA000A69EA680A85001010ABFF28E0001B86B34
:104BB000B76FB7C0B8F0B76BF2CF0AF1F29E130E21
:104BC000A96EA69CA69EA680A85001010ABFF28EDF
:104BD0000001B727000EB823F2CF0AF1F29E240E8F
:104BE000A96EA69CA69EA680A85001010ABFF28EBF
:104BF0000001BA6BB96FB9C0BAF0B96BF2CF0AF164
:104C0000F29E140EA96EA69CA69EA680A850010135
:104C10000ABFF28E0001B927000EBA23F2CF0AF1C3
:104C2000F29E250EA96EA69CA69EA680A850010104
:104C30000ABFF28E0001BC6BBB6FBBC0BCF0BB6B8C
:104C4000F2CF0AF1F29E150EA96EA69CA69EA68032
:104C5000A85001010ABFF28E0001BB27000EBC2341
:104C6000F2CF0AF1F29E260EA96EA69CA69EA68001
:104C7000A85001010ABFF28E0001BE6BBD6FBDC01E
:104C8000BEF0BD6BF2CF0AF1F29E160EA96EA69C85
:104C9000A69EA680A85001010ABFF28E0001BD2782
:104CA000000EBE23F2CF0AF1F29E270EA96EA69C3B
:104CB000A69EA680A85001010ABFF28E0001C06B1B
:104CC000BF6FBFC0C0F0BF6BF2CF0AF1F29E170EEC
:104CD000A96EA69CA69EA680A85001010ABFF28ECE
:104CE0000001BF27000EC02301010A6B0A51000119
:104CF000C8EC06F001010A2B0001CDEC11F0110EF9
:104D000001010A5DF3E1100EE96EB8C00BF1B7C006
:104D10000AF100011EEC14F001010A6B0A510001B6
:104D2000E0EC06F001010A2B0001CDEC11F0110EB0
:104D300001010A5DF3E1100EE96EB6C00BF1B5C0DA
:104D40000AF100011EEC14F001010A6B0A51000186
:104D5000F8EC06F001010A2B0001CDEC11F0110E68
:104D600001010A5DF3E1100EE96EB4C00BF1B3C0AE
:104D70000AF100011EEC14F001010A6B0A51000156
:104D800010EC07F001010A2B0001CDEC11F0110E1F
:104D900001010A5DF3E1100EE96EB2C00BF1B1C082
:104DA0000AF100011EEC14F001010A6B0A51000126
:104DB00028EC07F001010A2B0001CDEC11F0110ED7
:104DC00001010A5DF3E1100EE96EC0C00BF1BFC036
:104DD0000AF100011EEC14F001010A6B0A510001F6
:104DE00040EC07F001010A2B0001CDEC11F0110E8F
:104DF00001010A5DF3E1100EE96EBEC00BF1BDC00A
:104E00000AF100011EEC14F001010A6B0A510001C5
:104E100058EC07F001010A2B0001CDEC11F0110E46
:104E200001010A5DF3E1100EE96EBCC00BF1BBC0DD
:104E30000AF100011EEC14F001010A6B0A51000195
:104E400070EC07F001010A2B0001CDEC11F0110EFE
:104E500001010A5DF3E1100EE96EBAC00BF1B9C0B1
:104E60000AF100011EEC14F03D52D8A4ABD0C150A1
:104E7000C00B0B09C16EC090C082C084C08EC280BE
:104E8000100E016EC250C30B0110C26EC282C2B2BC
:104E9000FED7C3CF31F0C4CF32F0140E315E000E16
:104EA000325A32C00BF131C00AF173EF14F003C073
:104EB00026F102C025F101C024F100C023F1010157
:104EC0002A6B296B200E286F770E276F00018FEC5D
:104ED00014F000C00AF101C00BF102C00CF103C0D4
:104EE0000DF1D88203C026F102C025F101C024F1E2
:104EF00000C023F1520E01012A6FB80E296F2E0E49
:104F0000286F800E276F00010AEC15F000C00AF12F
:104F100001C00BF102C00CF103C00DF103C026F17A
:104F200002C025F101C024F100C023F101012A6B68
:104F3000296B480E286F850E276F00018FEC14F047
:104F400003C036F002C035F001C034F000C033F0C9
:104F5000660E0101266F256F246F7F0E236F36C00A
:104F60002AF135C029F134C028F133C027F10001FE
:104F70008FEC14F000C00AF101C00BF102C00CF17B
:104F800003C00DF1D89203C026F102C025F101C083
:104F900024F100C023F101012A6B296B286B840ED8
:104FA000276F00010AEC15F003C03AF002C039F097
:104FB00001C038F000C037F031C03CF0010132C010
:104FC0003BF00001010E3D263D506308D8A03D6A2C
:104FD000C150C00B0B09C16EC080C092C084C08E8E
:104FE000C280050E01010A6F000146EF16F0325033
:104FF0000308D8A097D004E131508408D8A092D0FB
:1050000032500008D8B08ED0FF0A04E13150DA08DF
:10501000D8B088D001010A6B0A51000188EC07F072
:1050200001010A2B0001CDEC11F00D0E01010A5D0A
:10503000F3E1010EE96E36C00DF135C00CF134C05C
:105040000BF133C00AF10E6F0001C1EC16F0430EF4
:10505000CDEC11F0200ECDEC11F0200ECDEC11F0C6
:10506000020EE96E3AC00DF139C00CF138C00BF1F7
:1050700037C00AF1010E01010E6F0001C1EC16F0FC
:105080001A0E01010A6F0A51000188EC07F00101B4
:105090000A2B0001CDEC11F01E0E01010A5DF3E1B7
:1050A000116B050E126F000138EC12F0020EE96E62
:1050B0003AC00DF139C00CF138C00BF137C00AF11C
:1050C00001010E6B000192EC17F08BEC18F0460E0C
:1050D0000101176F0001D6EC12F0200E0101176FCD
:1050E0000001D6EC12F0300E0101116F050E126FA7
:1050F000000138EC12F0010EE96E36C00DF135C03A
:105100000CF134C00BF133C00AF101010E6B000148
:1051100092EC17F08BEC18F0430E0101176F0001B1
:10512000D6EC12F0926B916B946B936B966B956BC4
:10513000986B976BD16B7751D15D02E178536CE03E
:105140008282040E016EC250C30B0110C26EC28275
:10515000C2B2FED7C3CF89F0C4CF8AF0020E0101DC
:105160000A6FFA0E0B6F0001AEEC18F001010A2F66
:10517000F8D7000E016EC250C30B0110C26EC2827E
:10518000C2B2FED7C4CF8CF00001C3CF8BF00A0EA1
:1051900001010B6F000106EC12F08292040E016E09
:1051A000C250C30B0110C26EC282C2B2FED7C3CFBF
:1051B0008DF0C4CF8EF0020E01010A6FFA0E0B6F54
:1051C0000001AEEC18F001010A2FF8D7000E016EB5
:1051D000C250C30B0110C26EC282C2B2FED7C4CF8E
:1051E00090F00001C3CF8FF00A0E01010B6F000198
:1051F00006EC12F0895191278A5192238B51932703
:105200008C5194238D5195278E5196238F5197273A
:1052100090519823D12B8FD792C00DF191C00CF1F2
:1052200078C00FF177C00EF1BFEC18F002C07AF031
:1052300001C079F096C00DF195C00CF178C00FF166
:1052400077C00EF1BFEC18F002C07EF001C07DF017
:1052500094C00DF193C00CF178C00FF177C00EF13E
:10526000BFEC18F002C07CF001C07BF098C00DF1DB
:1052700097C00CF178C00FF177C00EF1BFEC18F0B9
:1052800002C080F001C07FF07A51010805E303E11C
:105290007951900801E3E8D57E51010805E303E167
:1052A0007D51900801E3E0D57C51010805E303E15D
:1052B0007B51900801E3D8D58051010805E303E153
:1052C0007F51900801E3D0D5AF5306E1B05304E11C
:1052D000070EB06FD00EAF6FA95306E1AA5304E1D9
:1052E000070EAA6FD00EA96FA35306E1A45304E1E1
:1052F000070EA46FD00EA36F9D5306E19E5304E1E9
:10530000070E9E6FD00E9D6FAC517A5D09E303E1ED
:10531000AB51795D05E37AC0ACF079C0ABF00BD04E
:105320007A51B05D08E303E1AF51795D04E27AC0E0
:10533000B0F079C0AFF0A6517E5D09E303E1A5515D
:105340007D5D05E37EC0A6F07DC0A5F00BD07E514B
:10535000AA5D08E303E1A9517D5D04E27EC0AAF0E5
:105360007DC0A9F0A0517C5D09E303E19F517B5D05
:1053700005E37CC0A0F07BC09FF00BD07C51A45D06
:1053800008E303E1A3517B5D04E27CC0A4F07BC091
:10539000A3F09A51805D09E303E199517F5D05E334
:1053A00080C09AF07FC099F00BD080519E5D08E3D9
:1053B00003E19D517F5D04E280C09EF07FC09DF0BF
:1053C00001010A6B0A510001A5EC07F001010A2B4B
:1053D0000001CDEC11F0060E01010A5DF3E1100EA3
:1053E000E96E7AC00BF179C00AF100011EEC14F0ED
:1053F00001010A6B0A510001B7EC07F001010A2B09
:105400000001CDEC11F0060E01010A5DF3E1100E72
:10541000E96E7EC00BF17DC00AF100011EEC14F0B4
:1054200001010A6B0A510001C9EC07F001010A2BC6
:105430000001CDEC11F0060E01010A5DF3E1100E42
:10544000E96E7CC00BF17BC00AF100011EEC14F088
:1054500001010A6B0A510001DBEC07F001010A2B84
:105460000001CDEC11F0060E01010A5DF3E1100E12
:10547000E96E80C00BF17FC00AF100011EEC14F050
:10548000B8517A5D08E303E1B751795D04E37AC06E
:10549000B8F079C0B7F0B6517E5D08E303E1B551CD
:1054A0007D5D04E37EC0B6F07DC0B5F0B4517C5D97
:1054B00008E303E1B3517B5D04E37CC0B4F07BC03F
:1054C000B3F0B251805D08E303E1B1517F5D04E3C5
:1054D00080C0B2F07FC0B1F07951B75D01010A6FB1
:1054E00000017A51B85901010B6F0D6F0AC10CF11F
:1054F0000F6B640E0E6F0001E2EC18F002C00BF1AE
:1055000001C00AF102C00DF101C00CF1C0C00FF1E1
:10551000BFC00EF1BFEC18F002C082F001C081F0F4
:105520007D51B55D01010A6F00017E51B65901013F
:105530000B6F0D6F0AC10CF10F6B640E0E6F000143
:10554000E2EC18F002C00BF101C00AF102C00DF14B
:1055500001C00CF1BEC00FF1BDC00EF1BFEC18F0E0
:1055600002C086F001C085F07B51B35D01010A6F76
:1055700000017C51B45901010B6F0D6F0AC10CF190
:105580000F6B640E0E6F0001E2EC18F002C00BF11D
:1055900001C00AF102C00DF101C00CF1BCC00FF155
:1055A000BBC00EF1BFEC18F002C084F001C083F064
:1055B0007F51B15D01010A6F00018051B2590101B3
:1055C0000B6F0D6F0AC10CF10F6B640E0E6F0001B3
:1055D000E2EC18F002C00BF101C00AF102C00DF1BB
:1055E00001C00CF1BAC00FF1B9C00EF1BFEC18F058
:1055F00002C088F001C087F001010A6B0A51000166
:10560000EDEC07F001010A2B0001CDEC11F0070EC3
:1056100001010A5DF3E1100EE96E82C00BF181C059
:105620000AF100011EEC14F001010A6B0A5100019D
:1056300000EC08F001010A2B0001CDEC11F0070E7F
:1056400001010A5DF3E1100EE96E86C00BF185C021
:105650000AF100011EEC14F001010A6B0A5100016D
:1056600013EC08F001010A2B0001CDEC11F0070E3C
:1056700001010A5DF3E1100EE96E84C00BF183C0F5
:105680000AF100011EEC14F001010A6B0A5100013D
:1056900026EC08F001010A2B0001CDEC11F0070EF9
:1056A00001010A5DF3E1100EE96E88C00BF187C0BD
:1056B0000AF100011EEC14F0825303E18151C70886
:1056C00003E2826B010E816F865303E18551C708A7
:1056D00003E2866B010E856F845303E18351C70893
:1056E00003E2846B010E836F885303E18751C7087F
:1056F00003E2886B010E876F01010A6B0A510001FA
:10570000EDEC07F001010A2B0001CDEC11F0070EC2
:1057100001010A5DF3E1100EE96E82C00BF181C058
:105720000AF100011EEC14F001010A6B0A5100019C
:1057300000EC08F001010A2B0001CDEC11F0070E7E
:1057400001010A5DF3E1100EE96E86C00BF185C020
:105750000AF100011EEC14F001010A6B0A5100016C
:1057600013EC08F001010A2B0001CDEC11F0070E3B
:1057700001010A5DF3E1100EE96E84C00BF183C0F4
:105780000AF100011EEC14F001010A6B0A5100013C
:1057900026EC08F001010A2B0001CDEC11F0070EF8
:1057A00001010A5DF3E1100EE96E88C00BF187C0BC
:1057B0000AF100011EEC14F08151855DC16F825128
:1057C0008659C26F8751835DC36F88518459C46FF6
:1057D00001010A6B0A51000139EC08F001010A2BA2
:1057E0000001CDEC11F00E0E01010A5DF3E1100E87
:1057F000E96EC2C00BF1C1C00AF10001F3EC18F070
:10580000200ECDEC11F001010A6B0A51000150ECA1
:1058100008F001010A2B0001CDEC11F00E0E010180
:105820000A5DF3E1100EE96EC4C00BF1C3C00AF1CA
:105830000001F3EC18F0200ECDEC11F00D0ECDECC4
:1058400011F00A0ECDEC11F0D36B5A0ED26FD56B5E
:10585000D46FD76BD66FD96BD86FC15310E1C253D9
:105860000EE1C4BF0CD0C45303E1C351000807E2EA
:10587000E56BE46B070EE36F870EE26F29D0C1532F
:105880000BE1C25309E1C4AF07D0E56BE46B340E02
:10589000E36F850EE26F1CD0C2BF0ED0C25303E18E
:1058A000C151000809E2C35307E1C45305E1E56BA8
:1058B000E46BE36BE26B0CD0C2AF0AD0C35308E1D8
:1058C000C45306E1E56BE46B340EE36F860EE26FC2
:1058D000C2BFE8D0C25304E1C1510008D8B0E2D041
:1058E000C4BFE0D0C45304E1C3510008D8B0DAD03B
:1058F000C4C012F1C3C011F164EC19F000C00AF188
:1059000001C00BF102C00CF103C00DF1D3C012F1C4
:10591000D2C011F164EC19F00DC126F10CC125F1D2
:105920000BC124F10AC123F103C02AF102C029F1FD
:1059300001C028F100C027F18CEC19F003C0E1F0A0
:1059400002C0E0F001C0DFF000C0DEF0C2C012F122
:10595000C1C011F164EC19F000C00AF101C00BF1F3
:1059600002C00CF103C00DF1D5C012F1D4C011F189
:1059700064EC19F00DC126F10CC125F10BC124F125
:105980000AC123F103C02AF102C029F101C028F1A4
:1059900000C027F18CEC19F003C0DDF002C0DCF090
:1059A00001C0DBF000C0DAF0E1C026F1E0C025F173
:1059B000DFC024F1DEC023F1DDC02AF1DCC029F113
:1059C000DBC028F1DAC027F18CEC19F003C0F5F048
:1059D00002C0F4F001C0F3F000C0F2F0E1C026F123
:1059E000E0C025F1DFC024F1DEC023F1DDC02AF1E3
:1059F000DCC029F1DBC028F1DAC027F18CEC19F00A
:105A000000C00AF101C00BF102C00CF103C00DF19E
:105A100003C011F102C010F101C00FF100C00EF17E
:105A200078EC1AF000C00AF101C00BF102C00CF1D1
:105A300003C00DF103C026F102C025F101C024F11D
:105A400000C023F1E00E01012A6F2E0E296F650EB2
:105A5000286F840E276F00018FEC14F0EACF0BF152
:105A6000E9CF0AF1D8820101266B256B340E246F31
:105A7000870E236F03C02AF102C029F101C028F16B
:105A800000C027F100010AEC15F00BC1EAFF0AC1C2
:105A9000E9FF03C0E5F002C0E4F001C0E3F000C09C
:105AA000E2F0A7D1C2BFC9D0C25304E1C15100087E
:105AB000D8B0C3D0C4BF01D0C0D0C4C012F1C3C0DD
:105AC00011F164EC19F000C00AF101C00BF102C041
:105AD0000CF103C00DF1D7C012F1D6C011F164EC86
:105AE00019F00DC126F10CC125F10BC124F10AC139
:105AF00023F103C02AF102C029F101C028F100C03E
:105B000027F18CEC19F003C0E1F002C0E0F001C015
:105B1000DFF000C0DEF0C2C012F1C1C011F164ECD0
:105B200019F000C00AF101C00BF102C00CF103C072
:105B30000DF1D5C012F1D4C011F164EC19F00DC112
:105B400026F10CC125F10BC124F10AC123F103C0D8
:105B50002AF102C029F101C028F100C027F18CEC24
:105B600019F003C0DDF002C0DCF001C0DBF000C0C2
:105B7000DAF0E1C026F1E0C025F1DFC024F1DEC09B
:105B800023F1DDC02AF1DCC029F1DBC028F1DAC045
:105B900027F18CEC19F003C0F5F002C0F4F001C05D
:105BA000F3F000C0F2F0E1C026F1E0C025F1DFC063
:105BB00024F1DEC023F1DDC02AF1DCC029F1DBC015
:105BC00028F1DAC027F18CEC19F000C00AF101C00D
:105BD0000BF102C00CF103C00DF103C011F102C0C2
:105BE00010F101C00FF100C00EF178EC1AF000C006
:105BF0000AF101C00BF102C00CF103C00DF103C0AA
:105C000026F102C025F101C024F100C023F1E00E0D
:105C100001012A6F2E0E296F650E286F840E276FE3
:105C200000018FEC14F000C0E2F00150800AE36F35
:105C300002C0E4F003C0E5F0DCD0C2BF01D0D9D08F
:105C4000C4C012F1C3C011F164EC19F000C00AF134
:105C500001C00BF102C00CF103C00DF1D3C012F171
:105C6000D2C011F164EC19F00DC126F10CC125F17F
:105C70000BC124F10AC123F103C02AF102C029F1AA
:105C800001C028F100C027F18CEC19F003C0E1F04D
:105C900002C0E0F001C0DFF000C0DEF0C2C012F1CF
:105CA000C1C011F164EC19F000C00AF101C00BF1A0
:105CB00002C00CF103C00DF1D9C012F1D8C011F12E
:105CC00064EC19F00DC126F10CC125F10BC124F1D2
:105CD0000AC123F103C02AF102C029F101C028F151
:105CE00000C027F18CEC19F003C0DDF002C0DCF03D
:105CF00001C0DBF000C0DAF0E1C026F1E0C025F120
:105D0000DFC024F1DEC023F1DDC02AF1DCC029F1BF
:105D1000DBC028F1DAC027F18CEC19F003C0F5F0F4
:105D200002C0F4F001C0F3F000C0F2F0E1C026F1CF
:105D3000E0C025F1DFC024F1DEC023F1DDC02AF18F
:105D4000DCC029F1DBC028F1DAC027F18CEC19F0B6
:105D500000C00AF101C00BF102C00CF103C00DF14B
:105D600003C011F102C010F101C00FF100C00EF12B
:105D700078EC1AF000C00AF101C00BF102C00CF17E
:105D800003C00DF103C026F102C025F101C024F1CA
:105D900000C023F1E00E01012A6F2E0E296F650E5F
:105DA000286F840E276F00018FEC14F0EACF0BF1FF
:105DB000E9CF0AF1D8820101266B256B340E246FDE
:105DC000860E236F03C02AF102C029F101C028F119
:105DD00000C027F100010AEC15F00BC1EAFF0AC16F
:105DE000E9FF03C0E5F002C0E4F001C0E3F000C049
:105DF000E2F0360E0101116F126B000138EC12F067
:105E0000020EE96EE5C00DF1E4C00CF1E3C00BF148
:105E1000E2C00AF101010E6B00010BEF1DF08BECEB
:105E200018F001010A6B0A51000168EC08F0010149
:105E30000A2B0001CDEC11F00A0E01010A5DF3E11D
:105E4000020EE96EE5C00DF1E4C00CF1E3C00BF108
:105E5000E2C00AF10E6B0001C1EC16F0200ECDEC91
:105E600011F00A0ECDEC11F00D0ECDEC11F0E5C0E5
:105E7000EDF0E4C0ECF0E3C0EBF0E2C0EAF0EA6A77
:105E8000E60EE96EF2CF0AF1F29E000E7FEC08F00A
:105E90000A000900F550EE6E0009FBE101010ABF9E
:105EA000F28EEDC022F1ECC021F1EBC020F1EAC08E
:105EB0001FF19A0E266F990E256F310E246F820EF8
:105EC000236F00013BEC1AF01AE3EA6AE60EE96E72
:105ED000F2CF0AF1F29E000E8EEC08F00A000900E3
:105EE000F550EE6E0009FBE101010ABFF28E020ED1
:105EF0000A6F0001E9EC1DF092988988ECD2EDC0A0
:105F000022F1ECC021F1EBC020F1EAC01FF1330E09
:105F10000101266F256F070E246F840E236F000189
:105F20003BEC1AF01AE3EA6AE60EE96EF2CF0AF1E8
:105F3000F29E000E9DEC08F00A000900F550EE6E8E
:105F40000009FBE101010ABFF28E0A0E0A6F00018F
:105F5000E9EC1DF092988998BED2EDC022F1ECC018
:105F600021F1EBC020F1EAC01FF1330E0101266FD1
:105F7000256F610E246F840E236F00013BEC1AF035
:105F80001AE3EA6AE60EE96EF2CF0AF1F29E000E1B
:105F9000ACEC08F00A000900F550EE6E0009FBE1D8
:105FA00001010ABFF28E060E0A6F0001E9EC1DF036
:105FB0009298899890D2EDC022F1ECC021F1EBC00B
:105FC00020F1EAC01FF19A0E0101266F990E256F8C
:105FD0001D0E246F850E236F00013BEC1AF01AE3AF
:105FE000EA6AE60EE96EF2CF0AF1F29E000EBBEC11
:105FF00008F00A000900F550EE6E0009FBE101010E
:106000000ABFF28E0B0E0A6F0001E9EC1DF09298A8
:10601000899861D2EDC022F1ECC021F1EBC020F1F2
:10602000EAC01FF19A0E0101266F990E256F4A0EE4
:10603000246F850E236F00013BEC1AF01AE3EA6A25
:10604000E60EE96EF2CF0AF1F29E000ECAEC08F0FD
:106050000A000900F550EE6E0009FBE101010ABFDC
:10606000F28E050E0A6F0001E9EC1DF092988998F6
:1060700032D2EDC022F1ECC021F1EBC020F1EAC038
:106080001FF19A0E0101266F990E256F770E246F6E
:10609000850E236F00013BEC1AF01AE3EA6AE60E64
:1060A000E96EF2CF0AF1F29E000ED9EC08F00A0078
:1060B0000900F550EE6E0009FBE101010ABFF28E06
:1060C0000C0E0A6F0001E9EC1DF09298899803D23A
:1060D000EDC022F1ECC021F1EBC020F1EAC01FF1CC
:1060E000CD0E0101266F4C0E256F120E246F860E09
:1060F000236F00013BEC1AF01AE3EA6AE60EE96E40
:10610000F2CF0AF1F29E000EE8EC08F00A00090056
:10611000F550EE6E0009FBE101010ABFF28E070E99
:106120000A6F0001E9EC1DF092988998D4D1EDC076
:1061300022F1ECC021F1EBC020F1EAC01FF1CD0E3D
:106140000101266FCC0E256F280E246F860E236F5B
:1061500000013BEC1AF01AE3EA6AE60EE96EF2CFB0
:106160000AF1F29E000EF7EC08F00A000900F55063
:10617000EE6E0009FBE101010ABFF28E0D0E0A6FFF
:106180000001E9EC1DF092988998A5D1EDC022F1AB
:10619000ECC021F1EBC020F1EAC01FF1CD0E0101EE
:1061A000266F4C0E256F3F0E246F860E236F000165
:1061B0003BEC1AF01AE3EA6AE60EE96EF2CF0AF156
:1061C000F29E000E06EC09F00A000900F550EE6E92
:1061D0000009FBE101010ABFF28E030E0A6F000104
:1061E000E9EC1DF09298899876D1EDC022F1ECC0CF
:1061F00021F1EBC020F1EAC01FF1CD0E0101266FA5
:10620000CC0E256F550E246F860E236F00013BECDC
:106210001AF01AE3EA6AE60EE96EF2CF0AF1F29E8C
:10622000000E15EC09F00A000900F550EE6E0009A9
:10623000FBE101010ABFF28E0E0E0A6F0001E9ECCC
:106240001DF09298899847D1EDC022F1ECC021F160
:10625000EBC020F1EAC01FF1CD0E0101266F4C0EFC
:10626000256F6C0E246F860E236F00013BEC1AF035
:106270001AE3EA6AE60EE96EF2CF0AF1F29E000E28
:1062800024EC09F00A000900F550EE6E0009FBE16C
:1062900001010ABFF28E080E0A6F0001E9EC1DF041
:1062A0009298899818D1EDC022F1ECC021F1EBC091
:1062B00020F1EAC01FF1660E0101266F256F010E65
:1062C000246F870E236F00013BEC1AF01AE3EA6A91
:1062D000E60EE96EF2CF0AF1F29E000E33EC09F001
:1062E0000A000900F550EE6E0009FBE101010ABF4A
:1062F000F28E0F0E0A6F0001E9EC1DF0929889985A
:10630000EAD0EDC022F1ECC021F1EBC020F1EAC0EF
:106310001FF1660E0101266FA60E256F0C0E246F6D
:10632000870E236F00013BEC1AF01AE3EA6AE60ECF
:10633000E96EF2CF0AF1F29E000E42EC09F00A007B
:106340000900F550EE6E0009FBE101010ABFF28E73
:10635000040E0A6F0001E9EC1DF092988998BBD0F9
:10636000EDC022F1ECC021F1EBC020F1EAC01FF139
:10637000660E0101266FE60E256F170E246F870E3D
:10638000236F00013BEC1AF01AE3EA6AE60EE96EAD
:10639000F2CF0AF1F29E000E51EC09F00A0009005A
:1063A000F550EE6E0009FBE101010ABFF28E100EFE
:1063B0000A6F0001E9EC1DF0929889988CD0EDC02D
:1063C00022F1ECC021F1EBC020F1EAC01FF1660E12
:1063D0000101266F260E256F230E246F870E236F73
:1063E00000013BEC1AF01AE3EA6AE60EE96EF2CF1E
:1063F0000AF1F29E000E60EC09F00A000900F55067
:10640000EE6E0009FBE101010ABFF28E090E0A6F70
:106410000001E9EC1DF0929889985DD0EDC022F161
:10642000ECC021F1EBC020F1EAC01FF19A0E01018E
:10643000266F590E256F2E0E246F870E236F0001D5
:106440003BEC1AF01AE3EA6AE60EE96EF2CF0AF1C3
:10645000F29E000E6FEC09F00A000900F550EE6E96
:106460000009FBE101010ABFF28E110E0A6F000163
:10647000E9EC1DF0929889982ED0EDC022F1ECC085
:1064800021F1EBC020F1EAC01FF1CD0E0101266F12
:106490000C0E256F340E246F870E236F00013BEC2A
:1064A0001AF019E3EA6AE60EE96EF2CF0AF1F29EFB
:1064B000000E8EEC08F00A000900F550EE6E00099F
:1064C000FBE101010ABFF28E020E0A6F0001E9EC46
:1064D0001DF0929889883C0E0101116F020E126F17
:1064E000000138EC12F0EA6AE60EE96E000EEF10D9
:1064F00010E0EACF0BF1E9CF0AF1EFCF17F1D6ECBC
:1065000012F00BC1EAFF0AC1E9FFE92AD8B4EA2A6E
:10651000EDD7080E016EC250C30B0110C26E130EF0
:10652000006E002EFED700D0C282C2B2FED7C3CF0B
:10653000C9F0C4CFCAF00C0E016EC250C30B0110DB
:10654000C26E130E006E002EFED700D0C282C2B201
:10655000FED7C3CFCBF0C4CFCCF022EF1FF042EF79
:106560001FF0F40EC95D01010A6F010E0001CA5946
:1065700001010B6F036A0001D051006EE8BE0306F3
:1065800001010A5F03500B5B0BC112F10AC111F14B
:10659000000164EC19F003C026F102C025F101C02E
:1065A00024F100C023F101012A6B296B400E286FF2
:1065B0007F0E276F00018FEC14F003C014F102C0AE
:1065C00013F101C012F100C011F17FEC1FF001C006
:1065D000CDF0F40ECB5D01010A6F010E0001CC5924
:1065E00001010B6F036A0001CF51006EE8BE030684
:1065F00001010A5F03500B5B0BC112F10AC111F1DB
:10660000000164EC19F003C026F102C025F101C0BD
:1066100024F100C023F101012A6B296B400E286F81
:106620007F0E276F00018FEC14F003C014F102C03D
:1066300013F101C012F100C011F17FEC1FF001C095
:10664000CEF0CD51800A260803E3A60ECD6F07D009
:10665000CDBF05D0CD51590802E25A0ECD6FCE51B3
:10666000800A260803E3A60ECE6F07D0CEBF05D062
:10667000CE51590802E25A0ECE6F0101116B040E81
:10668000126F000138EC12F0CDC00AF1130E0101B7
:106690000B6F00019DEC1FF03C0E0101116F040E09
:1066A000126F000138EC12F0CEC00AF1130E010196
:1066B0000B6F00019DEC1FF001010A6B0A510001F4
:1066C0007EEC09F001010A2B0001CDEC11F00A0E5D
:1066D00001010A5DF3E1CDC00AF1130E0B6F000159
:1066E00012EC20F0200ECDEC11F00A0ECDEC11F0E2
:1066F0000D0ECDEC11F001010A6B0A51000194EC72
:1067000009F001010A2B0001CDEC11F00A0E010184
:106710000A5DF3E1CEC00AF1130E0B6F000112EC1B
:1067200020F00D0E01010A6F0A51000194EC09F0EE
:1067300001010A2B0001CDEC11F0130E01010A5DDD
:10674000F3E1CDC00AF100019DEF20F0CEC00AF1C7
:1067500033EF22F0EDC014F1ECC013F1EBC012F1F5
:10676000EAC011F17FEC1FF0F16BF06B02C0EFF0AB
:1067700001C0EEF0EEC0C5F0EFC0EEF0F0C0EFF0FB
:10678000F1C0F0F0F16BEEC0C6F0EFC0EEF0F0C07B
:10679000EFF0F1C0F0F0F16BEEC0C7F0EFC0EEF03B
:1067A000F0C0EFF0F1C0F0F0F16BEEC0C8F03BC00C
:1067B000FEF03CC0FDF0CEC0FCF0CDC0FBF0C8C088
:1067C000FAF0C7C0F9F0C6C0F8F0C5C0F7F006ECA3
:1067D00014F07AEC23F077EC23F001521EE0010E66
:1067E000616F606B5F6A030E5E6E3BC05DF03CC024
:1067F0005CF0CEC05BF0CDC05AF0010E01010A6F13
:106800000C6B5A0E0B6F0E6B080E0D6F020E0F6F96
:106810000001D0EC23F0015200E0010E01010B6FEA
:10682000000106EC12F006EC14F07AEC23F077ECA1
:1068300023F0015260E0010E616F606B5F6A040E2D
:106840005E6EC8C05DF0C7C05CF0C6C05BF0C5C07E
:106850005AF0010E01010A6F0C6B5A0E0B6F0E6B92
:10686000080E0D6F020E0F6F0001D0EC23F00152E5
:1068700000E0010E01010A6F000127EF24F0015230
:1068800039E0010E01010A6F0C6B620E0B6F0E6B8B
:10689000020E0D6F0001AAEF24F001010A6B0A51EC
:1068A0000001ABEC09F001010A2B0001CDEC11F065
:1068B000170E01010A5DF3E162C00AF1370E0B6F9A
:1068C0000001CFEC24F0200ECDEC11F0300ECDEC19
:1068D00011F0780ECDEC11F063C00AF1370E010112
:1068E0000B6F0001CFEC24F0625301E000D0635342
:1068F00001E000D0760781A4E9EF38F0F40EC95D1D
:10690000006E010ECA5900C0D0F0F40ECB5D006ECF
:10691000010ECC5900C0CFF0010EA96ED0C0A8FF67
:10692000A69CA69EA684F2CF00F0F29E0F01550E03
:10693000A76EAA0EA76EA682A6B2FED7A694005096
:10694000F212020EA96ECFC0A8FFA69CA69EA68436
:10695000F2CF00F0F29E550EA76EAA0EA76EA68289
:10696000A6B2FED7A6940050F212080E01010A6FDB
:10697000FA0E0B6F000106EC12F001010A2FF8D796
:1069800081A4E8EF38F00A6B0A510001C8EC09F065
:1069900001010A2B0001CDEC11F0150E01010A5D79
:1069A000F3E10D0E0001CDEC11F00A0ECDEC11F06B
:1069B000350ECDEC11F0040E01010A6FFA0E0B6FCB
:1069C000000106EC12F001010A2FF8D7340E000185
:1069D000CDEC11F0040E01010A6FFA0E0B6F0001ED
:1069E00006EC12F001010A2FF8D7330E0001CDECAE
:1069F00011F0040E01010A6FFA0E0B6F000106EC94
:106A000012F001010A2FF8D7320E0001CDEC11F07F
:106A1000040E01010A6FFA0E0B6F000106EC12F072
:106A200001010A2FF8D7310E0001CDEC11F0040E50
:106A300001010A6FFA0E0B6F000106EC12F0010162
:106A40000A2FF8D781A4C4D300019D51995D9B6F93
:106A50009E519A599C6FA3519F5DA16FA451A0595B
:106A6000A26FA951A55DA76FAA51A659A86FAF51F2
:106A7000AB5DAD6FB051AC59AE6F01010A6B0A51FD
:106A80000001E0EC09F001010A2B0001CDEC11F04E
:106A90000B0E01010A5DF3E1100EE96EACC00BF1C3
:106AA000ABC00AF100011EEC14F001010A6B0A519F
:106AB0000001F5EC09F001010A2B0001CDEC11F009
:106AC0000B0E01010A5DF3E1100EE96EA6C00BF199
:106AD000A5C00AF100011EEC14F001010A6B0A5175
:106AE00000010AEC0AF001010A2B0001CDEC11F0C3
:106AF0000B0E01010A5DF3E1100EE96EA0C00BF16F
:106B00009FC00AF100011EEC14F001010A6B0A514A
:106B100000011FEC0AF001010A2B0001CDEC11F07D
:106B20000B0E01010A5DF3E1100EE96E9AC00BF144
:106B300099C00AF100011EEC14F001010A6B0A5120
:106B4000000134EC0AF001010A2B0001CDEC11F038
:106B50000B0E01010A5DF3E1100EE96EAEC00BF100
:106B6000ADC00AF100011EEC14F001010A6B0A51DC
:106B7000000149EC0AF001010A2B0001CDEC11F0F3
:106B80000B0E01010A5DF3E1100EE96EA8C00BF1D6
:106B9000A7C00AF100011EEC14F001010A6B0A51B2
:106BA00000015EEC0AF001010A2B0001CDEC11F0AE
:106BB0000B0E01010A5DF3E1100EE96EA2C00BF1AC
:106BC000A1C00AF100011EEC14F001010A6B0A5188
:106BD000000173EC0AF001010A2B0001CDEC11F069
:106BE0000B0E01010A5DF3E1100EE96E9CC00BF182
:106BF0009BC00AF100011EEC14F099C00AF10101DA
:106C00000B6B100EA96E99C0A8FFA69CA69EA68429
:106C1000F2CF00F0F29E0F01550EA76EAA0EA76EDE
:106C2000A682A6B2FED7A6940050F2129AC00AF12C
:106C300001010B6B200EA96E9AC0A8FFA69CA69E10
:106C4000A684F2CF00F0F29E0F01550EA76EAA0E99
:106C5000A76EA682A6B2FED7A6940050F2129FC0DD
:106C60000AF101010B6B110EA96E9FC0A8FFA69C33
:106C7000A69EA684F2CF00F0F29E0F01550EA76EDD
:106C8000AA0EA76EA682A6B2FED7A6940050F21254
:106C9000A0C00AF101010B6B210EA96EA0C0A8FFD4
:106CA000A69CA69EA684F2CF00F0F29E0F01550E80
:106CB000A76EAA0EA76EA682A6B2FED7A694005013
:106CC000F212A5C00AF101010B6B120EA96EA5C04C
:106CD000A8FFA69CA69EA684F2CF00F0F29E0F010C
:106CE000550EA76EAA0EA76EA682A6B2FED7A694D0
:106CF0000050F212A6C00AF101010B6B220EA96E20
:106D0000A6C0A8FFA69CA69EA684F2CF00F0F29E85
:106D10000F01550EA76EAA0EA76EA682A6B2FED7C9
:106D2000A6940050F212ABC00AF101010B6B130ED6
:106D3000A96EABC0A8FFA69CA69EA684F2CF00F0C9
:106D4000F29E0F01550EA76EAA0EA76EA682A6B2DE
:106D5000FED7A6940050F212ACC00AF101010B6BF1
:106D6000230EA96EACC0A8FFA69CA69EA684F2CF57
:106D700000F0F29E0F01550EA76EAA0EA76EA68216
:106D8000A6B2FED7A6940050F2129BC00AF10101F0
:106D90000B6B140EA96E9BC0A8FFA69CA69EA68492
:106DA000F2CF00F0F29E0F01550EA76EAA0EA76E4D
:106DB000A682A6B2FED7A6940050F2129CC00AF199
:106DC00001010B6B240EA96E9CC0A8FFA69CA69E79
:106DD000A684F2CF00F0F29E0F01550EA76EAA0E08
:106DE000A76EA682A6B2FED7A6940050F212A1C04A
:106DF0000AF101010B6B150EA96EA1C0A8FFA69C9C
:106E0000A69EA684F2CF00F0F29E0F01550EA76E4B
:106E1000AA0EA76EA682A6B2FED7A6940050F212C2
:106E2000A2C00AF101010B6B250EA96EA2C0A8FF3A
:106E3000A69CA69EA684F2CF00F0F29E0F01550EEE
:106E4000A76EAA0EA76EA682A6B2FED7A694005081
:106E5000F212A7C00AF101010B6B160EA96EA7C0B2
:106E6000A8FFA69CA69EA684F2CF00F0F29E0F017A
:106E7000550EA76EAA0EA76EA682A6B2FED7A6943E
:106E80000050F212A8C00AF101010B6B260EA96E88
:106E9000A8C0A8FFA69CA69EA684F2CF00F0F29EF2
:106EA0000F01550EA76EAA0EA76EA682A6B2FED738
:106EB000A6940050F212ADC00AF101010B6B170E3F
:106EC000A96EADC0A8FFA69CA69EA684F2CF00F036
:106ED000F29E0F01550EA76EAA0EA76EA682A6B24D
:106EE000FED7A6940050F212AEC00AF101010B6B5E
:106EF000270EA96EAEC0A8FFA69CA69EA684F2CFC0
:106F000000F0F29E0F01550EA76EAA0EA76EA68284
:106F1000A6B2FED7A6940050F212F2CF0AF1F29E6A
:106F2000200EA96EA69CA69EA680A85001010ABFAD
:106F3000F28E0001B26BB16FB1C0B2F0B16BF2CFA3
:106F40000AF1F29E100EA96EA69CA69EA680A850DD
:106F500001010ABFF28E0001B127000EB223F2CF69
:106F60000AF1F29E210EA96EA69CA69EA680A850AC
:106F700001010ABFF28E0001B46BB36FB3C0B4F06D
:106F8000B36BF2CF0AF1F29E110EA96EA69CA69EDB
:106F9000A680A85001010ABFF28E0001B327000E9F
:106FA000B423F2CF0AF1F29E220EA96EA69CA69EF1
:106FB000A680A85001010ABFF28E0001B66BB56F22
:106FC000B5C0B6F0B56BF2CF0AF1F29E120EA96E03
:106FD000A69CA69EA680A85001010ABFF28E0001C1
:106FE000B527000EB623F2CF0AF1F29E230EA96E4A
:106FF000A69CA69EA680A85001010ABFF28E0001A1
:10700000B86BB76FB7C0B8F0B76BF2CF0AF1F29EAA
:10701000130EA96EA69CA69EA680A85001010ABFC9
:10702000F28E0001B727000EB823F2CF0AF1F29ECC
:10703000240EA96EA69CA69EA680A85001010ABF98
:10704000F28E0001BA6BB96FB9C0BAF0B96BF2CF6A
:107050000AF1F29E140EA96EA69CA69EA680A850C8
:1070600001010ABFF28E0001B927000EBA23F2CF48
:107070000AF1F29E250EA96EA69CA69EA680A85097
:1070800001010ABFF28E0001BC6BBB6FBBC0BCF03C
:10709000BB6BF2CF0AF1F29E150EA96EA69CA69EBE
:1070A000A680A85001010ABFF28E0001BB27000E86
:1070B000BC23F2CF0AF1F29E260EA96EA69CA69ED4
:1070C000A680A85001010ABFF28E0001BE6BBD6F01
:1070D000BDC0BEF0BD6BF2CF0AF1F29E160EA96ED6
:1070E000A69CA69EA680A85001010ABFF28E0001B0
:1070F000BD27000EBE23F2CF0AF1F29E270EA96E25
:10710000A69CA69EA680A85001010ABFF28E00018F
:10711000C06BBF6FBFC0C0F0BF6BF2CF0AF1F29E71
:10712000170EA96EA69CA69EA680A85001010ABFB4
:10713000F28E0001BF27000EC02301010A6B0A5125
:10714000000188EC0AF001010A2B0001CDEC11F0DE
:107150000F0E01010A5DF3E192988998C80E0B6F3A
:10716000000106EC12F092988988C80E01010B6F9D
:10717000000106EC12F092988998C80E01010B6F7D
:10718000000106EC12F092988988C80E01010B6F7D
:10719000000106EC12F092988998C80E01010B6F5D
:1071A000000106EC12F092988988C80E01010B6F5D
:1071B000000106EC12F092988998140E01010A6FF2
:1071C000FA0E0B6F000106EC12F001010A2FF8D73E
:1071D000000181A204D0786B020E776F06D0786B25
:1071E000010E776F2A0ECDEC11F034EF27F003007B
:020000040030CA
:0E00000000051E1F008381000FC00FE00F409F
:00000001FF
